     1                                  
     2                                  ; Public Domain
     3                                  
     4                                  ; test install command: install; .; useparat uninstall
     5                                  ; test run command: ; .; .
     6                                  
     7                                  %include "lmacros3.mac"
     1                              <1> [list -]
    14                              <2> [list -]
    14                              <1> [list -]
     8                                  %include "eld.mac"
     1                              <1> %if 0
     2                              <1> 
     3                              <1> Extensions for lDebug macros
     4                              <1> 
     5                              <1> Copyright (C) 2008-2025 E. C. Masloch
     6                              <1> 
     7                              <1> Usage of the works is permitted provided that this
     8                              <1> instrument is retained with the works, so that any entity
     9                              <1> that uses the works is notified of this instrument.
    10                              <1> 
    11                              <1> DISCLAIMER: THE WORKS ARE WITHOUT WARRANTY.
    12                              <1> 
    13                              <1> %endif
    14                              <1> 
    15                              <1> %ifndef ELD_MAC
    16                              <1> %define ELD_MAC 1
    17                              <1> 
    18                              <1> %include "lmacros3.mac"
     1                              <2> [list -]
    19                              <1> 
    20                              <1> 		; ELD executable header
    21                              <1> 	struc ELD_HEADER
    22 00000000 ????????            <1> eldhSignature:		resb 4	; "ELD1"
    23 00000004 ??????              <1> 			resb 3	; reserved
    24 00000007 ??                  <1> 			resb 1	; 26 (Ctrl-Z)
    25 00000008 ????????            <1> eldhCodeOffset:		resd 1	; position displacement from eldhSignature
    26 0000000C ????                <1> eldhCodeImageLength:	resw 1	; amount bytes, at least 32
    27 0000000E ????                <1> eldhCodeAllocLength:	resw 1	; amount bytes, added to prior. sum < 64 KiB
    28 00000010 ????????            <1> eldhDataOffset:		resd 1
    29 00000014 ????                <1> eldhDataImageLength:	resw 1	; (zero allowed)
    30 00000016 ????                <1> eldhDataAllocLength:	resw 1	; (zero allowed)
    31 00000018 ????                <1> eldhCodeEntrypoint:	resw 1	; within code section, used as displacement
    32 0000001A ????????            <1> eldhReserved:		resb 4	; reserved
    33 0000001E ????                <1> eldhExtensionSize:	resw 1	; from eldhSignature, -> past eldhx fields in use
    34                              <1> 	endstruc
    35                              <1> 	endarea ELD_HEADER, 1
    36                              <1> 
    37                              <1> 	struc ELD_HEADERX
    38 00000000 <res 20h>           <1> eldhxHeader:		resb ELD_HEADER_size
    39 00000020 ????????            <1> eldhxDescriptionOffset:	resd 1	; zero if none, from eldhxHeader. <= 128 Bytes
    40 00000024 ????????            <1> eldhxHelpOffset:	resd 1	; zero if none, from eldhxHeader
    41 00000028 ????????            <1> eldhxLibTable:		resd 1	; zero if none, from eldhxHeader
    42 0000002C ????????            <1> eldhxDateTimeOffset:	resd 1	; zero if none, from eldhxHeader
    43                              <1> 	alignb 16
    44                              <1> 	endstruc
    45                              <1> 
    46                              <1> 	struc ELD_TRAILER_HEADER
    47 00000000 ????????????????    <1> eldthSignature:		resb 8	; "ELD1TAIL"
    48 00000008 ????????            <1> eldthHeaderOffset:	resd 1	; negative displacement from eldthSignature,
    49                              <1> 				;  add this dword to the seek offset
    50 0000000C ????                <1> eldthReserved:		resw 1	; reserved, must be initialised to zero
    51 0000000E ????                <1> eldthChecksum:		resw 1	; sum of all words in trailer header = 0
    52                              <1> 	endstruc
    53                              <1> 	endarea ELD_TRAILER_HEADER, 1
    54                              <1> 
    55                              <1> 	struc ELD_LIBTABLE
    56 00000000 ????                <1> eldltFormat:		resw 1
    57                              <1> 	; 0 = uncompressed
    58                              <1> 	; 2 = heatshrink compressed
    59                              <1> 	; 3 = lzexedat -4 compressed
    60                              <1> 	; 4 = lzexedat -4 -l compressed
    61 00000002 ????                <1> eldltAmount:		resw 1
    62 00000004 ????????            <1> eldltOffset:		resd 1	; from eldhxHeader
    63                              <1> eldltCompressedLength:		; (dword, only present if format 2, 3, or 4)
    64                              <1> 	endstruc
    65                              <1> 	endarea ELD_LIBTABLE, 1
    66                              <1> 
    67                              <1> 		; ELD instance header
    68                              <1> 	struc ELD_INSTANCE
    69 00000000 ????                <1> eldiStartCode:		resw 1	; -> this structure itself (para aligned)
    70 00000002 ????                <1> eldiEndCode:		resw 1	; -> behind memory used by instance (para aligned)
    71 00000004 ????                <1> eldiStartData:		resw 1	; -> data in data entry section (para aligned), or 0
    72 00000006 ????                <1> eldiEndData:		resw 1	; -> behind data (para aligned), or 0
    73 00000008 ????????????????    <1> eldiIdentifier:		resb 8	; blank-filled text
    74 00000010 ????                <1> eldiFlags:		resw 1	; flags
    75                              <1> eldiListing_size equ 14
    76 00000012 <res Eh>            <1> eldiListing:		resb eldiListing_size
    77                              <1> 				; ASCIZ listing file name
    78                              <1> 	endstruc
    79                              <1> 		; flags for eldiFlags:
    80                              <1> eldifResident:		equ 1
    81                              <1> 
    82                              <1> 		; ELD link info header
    83                              <1> 	struc ELD_LINKINFO
    84 00000000 ????                <1> eldlSignature:		resw 1	; 0E1D1h
    85 00000002 ????????            <1> eldlReserved:		resw 2
    86 00000006 ????                <1> eldlUseLinkHash:	resw 1
    87 00000008 ????                <1> eldlDataAmount:		resw 1
    88 0000000A ????                <1> eldlDataPrefixes:	resw 1
    89 0000000C ????                <1> eldlDataEntries:	resw 1
    90 0000000E ????                <1> eldlDataAddresses:	resw 1
    91 00000010 ????                <1> eldlCodeAmount:		resw 1
    92 00000012 ????                <1> eldlCodePrefixes:	resw 1
    93 00000014 ????                <1> eldlCodeEntries:	resw 1
    94 00000016 ????                <1> eldlCodeAddresses:	resw 1
    95                              <1> 	endstruc
    96                              <1> 
    97                              <1> 	numdef ELD_CODE_VSTART, 9001h
    98                              <1> 	numdef ELD_DATA_VSTART, 8000h
    99                              <1> 	numdef ELD_RELOC_VSTART, 8000h
   100                              <1> 
   101                              <1> 	numdef ELD_RECLAIM_HINT, 0
   102                              <1> 	strdef ELD_LISTING, ""
   103                              <1> 	numdef ELD_DATETIME, 0
   104                              <1> 
   105                              <1> %if _ELD_DATETIME
   106                              <1>  %define PUT_ELDHX_DATETIME_OFFSET at eldhxDateTimeOffset, dd DATAOFFSET + datetime - datastart
   107                              <1>  %macro PUT_ELD_DATETIME 0.nolist
   108                              <1> datetime:	asciz __UTC_DATE__,'T',__UTC_TIME__,'Z'
   109                              <1> 		asciz		; for future extension
   110                              <1>  %endmacro
   111                              <1> %else
   112                              <1>  %define PUT_ELDHX_DATETIME_OFFSET
   113                              <1>  %define PUT_ELD_DATETIME
   114                              <1> %endif
   115                              <1> 
   116                              <1> %endif
     9                                  %include "eldcall.mac"
     1                              <1> %if 0
     2                              <1> 
     3                              <1> Extensions for lDebug call macros
     4                              <1> 
     5                              <1> Copyright (C) 2008-2024 E. C. Masloch
     6                              <1> 
     7                              <1> Usage of the works is permitted provided that this
     8                              <1> instrument is retained with the works, so that any entity
     9                              <1> that uses the works is notified of this instrument.
    10                              <1> 
    11                              <1> DISCLAIMER: THE WORKS ARE WITHOUT WARRANTY.
    12                              <1> 
    13                              <1> %endif
    14                              <1> 
    15                              <1> %ifndef ELDCALL_MAC
    16                              <1> %define ELDCALL_MAC 1
    17                              <1> 
    18                              <1> %include "lmacros3.mac"
     1                              <2> [list -]
    19                              <1> %include "nasmhash.mac"
     1                              <2> 
     2                              <2> %if 0
     3                              <2> 
     4                              <2> Hashing macros
     5                              <2>  by E. C. Masloch, 2019
     6                              <2> 
     7                              <2> Usage of the works is permitted provided that this
     8                              <2> instrument is retained with the works, so that any entity
     9                              <2> that uses the works is notified of this instrument.
    10                              <2> 
    11                              <2> DISCLAIMER: THE WORKS ARE WITHOUT WARRANTY.
    12                              <2> 
    13                              <2> %endif
    14                              <2> 
    15                              <2> %ifndef __NASMHASH_MAC__
    16                              <2> %assign __NASMHASH_MAC__ 1
    17                              <2> 
    18                              <2> 
    19                              <2> 	%macro hashdef 2+.nolist
    20                              <2> %ifempty %2
    21                              <2>  %assign _%1 1
    22                              <2> %else
    23                              <2> %ifstr %2
    24                              <2>  %define %%string %2
    25                              <2> %elifid %2
    26                              <2>  %defstr %%string %2
    27                              <2> %elifnum %2
    28                              <2>  %defstr %%string %2
    29                              <2> %eliftok %2
    30                              <2>  %defstr %%string %2
    31                              <2> %else
    32                              <2>  %error Unknown input
    33                              <2> %endif
    34                              <2> %strlen %%length %%string
    35                              <2> %assign %%hash 1
    36                              <2> %assign %%index 1
    37                              <2> %rep %%length
    38                              <2>  %substr %%char %%string %%index
    39                              <2>  %assign %%hash (%%hash * 31 + %%char) & 0FFFFh
    40                              <2>  %assign %%index %%index + 1
    41                              <2> %endrep
    42                              <2> %assign _%1 %%hash
    43                              <2> %endif
    44                              <2> 	%endmacro
    45                              <2> 
    46                              <2> 
    47                              <2> %endif
    20                              <1> %include "elddata.mac"
     1                              <2> %if 0
     2                              <2> 
     3                              <2> Extensions for lDebug data relocation macros
     4                              <2> 
     5                              <2> Copyright (C) 2008-2024 E. C. Masloch
     6                              <2> 
     7                              <2> Usage of the works is permitted provided that this
     8                              <2> instrument is retained with the works, so that any entity
     9                              <2> that uses the works is notified of this instrument.
    10                              <2> 
    11                              <2> DISCLAIMER: THE WORKS ARE WITHOUT WARRANTY.
    12                              <2> 
    13                              <2> %endif
    14                              <2> 
    15                              <2> %ifndef ELDDATA_MAC
    16                              <2> %define ELDDATA_MAC 1
    17                              <2> 
    18                              <2> %include "lmacros3.mac"
     1                              <3> [list -]
    19                              <2> %include "nasmhash.mac"
     1                              <3> 
     2                              <3> %if 0
     3                              <3> 
     4                              <3> Hashing macros
     5                              <3>  by E. C. Masloch, 2019
     6                              <3> 
     7                              <3> Usage of the works is permitted provided that this
     8                              <3> instrument is retained with the works, so that any entity
     9                              <3> that uses the works is notified of this instrument.
    10                              <3> 
    11                              <3> DISCLAIMER: THE WORKS ARE WITHOUT WARRANTY.
    12                              <3> 
    13                              <3> %endif
    14                              <3> 
    15                              <3> %ifndef __NASMHASH_MAC__
    16                              <3> %assign __NASMHASH_MAC__ 1
    17                              <3> 
    18                              <3> 
    19                              <3> 	%macro hashdef 2+.nolist
    20                              <3> %ifempty %2
    21                              <3>  %assign _%1 1
    22                              <3> %else
    23                              <3> %ifstr %2
    24                              <3>  %define %%string %2
    25                              <3> %elifid %2
    26                              <3>  %defstr %%string %2
    27                              <3> %elifnum %2
    28                              <3>  %defstr %%string %2
    29                              <3> %eliftok %2
    30                              <3>  %defstr %%string %2
    31                              <3> %else
    32                              <3>  %error Unknown input
    33                              <3> %endif
    34                              <3> %strlen %%length %%string
    35                              <3> %assign %%hash 1
    36                              <3> %assign %%index 1
    37                              <3> %rep %%length
    38                              <3>  %substr %%char %%string %%index
    39                              <3>  %assign %%hash (%%hash * 31 + %%char) & 0FFFFh
    40                              <3>  %assign %%index %%index + 1
    41                              <3> %endrep
    42                              <3> %assign _%1 %%hash
    43                              <3> %endif
    44                              <3> 	%endmacro
    45                              <3> 
    46                              <3> 
    47                              <3> %endif
    20                              <2> %include "eldcheck.mac"
     1                              <3> %if 0
     2                              <3> 
     3                              <3> Extensions for lDebug relocation check macros
     4                              <3> 
     5                              <3> Copyright (C) 2008-2023 E. C. Masloch
     6                              <3> 
     7                              <3> Usage of the works is permitted provided that this
     8                              <3> instrument is retained with the works, so that any entity
     9                              <3> that uses the works is notified of this instrument.
    10                              <3> 
    11                              <3> DISCLAIMER: THE WORKS ARE WITHOUT WARRANTY.
    12                              <3> 
    13                              <3> %endif
    14                              <3> 
    15                              <3> %ifndef ELDCHECK_MAC
    16                              <3> %define ELDCHECK_MAC 1
    17                              <3> 
    18                              <3> %assign ELDSTRICT 0
    19                              <3> %assign ELDSTRICTCOUNTER 0
    20                              <3> 
    21                              <3> 	%imacro eldstrict 1.nolist
    22                              <3> %ifidni %1, on
    23                              <3>  %assign ELDSTRICT 1
    24                              <3>  [warning +error=reloc-abs]
    25                              <3>  [warning +reloc-abs]
    26                              <3> %elifidni %1, off
    27                              <3>  %assign ELDSTRICT 0
    28                              <3>  [warning -reloc-abs]
    29                              <3> %else
    30                              <3>  %error Unknown keyword
    31                              <3> %endif
    32                              <3> 	%endmacro
    33                              <3> 
    34                              <3> 	%imacro reloc 1+.nolist
    35                              <3> %if ELDSTRICT
    36                              <3>  %if ELDSTRICTCOUNTER
    37                              <3>   %error Missing relocation
    38                              <3>  %endif
    39                              <3>  [warning -reloc-abs]
    40                              <3>  %assign ELDSTRICTCOUNTER 1
    41                              <3> %endif
    42                              <3> %1
    43                              <3> 	%endmacro
    44                              <3> 
    45                              <3> 	%imacro reloc2 1+.nolist
    46                              <3> %if ELDSTRICT
    47                              <3>  %if ELDSTRICTCOUNTER
    48                              <3>   %error Missing relocation
    49                              <3>  %endif
    50                              <3>  [warning -reloc-abs]
    51                              <3>  %assign ELDSTRICTCOUNTER 2
    52                              <3> %endif
    53                              <3> %1
    54                              <3> 	%endmacro
    55                              <3> 
    56                              <3> 	%imacro eldstrictcheck 0.nolist
    57                              <3> %if ELDSTRICT
    58                              <3>  %ifn ELDSTRICTCOUNTER
    59                              <3>   %error Unexpected relocation
    60                              <3>  %else
    61                              <3>   %assign ELDSTRICTCOUNTER ELDSTRICTCOUNTER - 1
    62                              <3>   %ifn ELDSTRICTCOUNTER
    63                              <3>    [warning +reloc-abs]
    64                              <3>   %endif
    65                              <3>  %endif
    66                              <3> %endif
    67                              <3> 	%endmacro
    68                              <3> 
    69                              <3> %endif
    70                              <3> 
    21                              <2> 
    22                              <2> 
    23                              <2> %assign ELDLINKER 0
    24                              <2> 
    25                              <2> %define INTERNAL_CODE_TO_CODE_RELOCATIONS ""
    26                              <2> %define INTERNAL_CODE_TO_DATA_RELOCATIONS ""
    27                              <2> %define INTERNAL_DATA_TO_CODE_RELOCATIONS ""
    28                              <2> %define INTERNAL_DATA_TO_DATA_RELOCATIONS ""
    29                              <2> %define INTERNAL_LINKER_CODE_TO_CODE_RELOCATIONS ""
    30                              <2> %define INTERNAL_LINKER_CODE_TO_DATA_RELOCATIONS ""
    31                              <2> %define INTERNAL_LINKER_DATA_TO_CODE_RELOCATIONS ""
    32                              <2> %define INTERNAL_LINKER_DATA_TO_DATA_RELOCATIONS ""
    33                              <2> %assign ELDDATA_OPTIONAL_STATUS 0		; not any seen yet
    34                              <2> %assign ELDDATA_PMREQUIRED_STATUS 0		; not any seen yet
    35                              <2> 
    36                              <2> 	%imacro internalcoderelocation 0-1.nolist -2
    37                              <2> %assign %%entry $ + _CURRENT_SECTION %+ FIXUP + %1
    38                              <2> %if ELDLINKER
    39                              <2>  %ifidni _CURRENT_SECTION_TYPE, DATA
    40                              <2>   %xdefine INTERNAL_LINKER_DATA_TO_CODE_RELOCATIONS INTERNAL_LINKER_DATA_TO_CODE_RELOCATIONS, %%entry
    41                              <2>  %else
    42                              <2>   %xdefine INTERNAL_LINKER_CODE_TO_CODE_RELOCATIONS INTERNAL_LINKER_CODE_TO_CODE_RELOCATIONS, %%entry
    43                              <2>  %endif
    44                              <2> %else
    45                              <2>  %ifidni _CURRENT_SECTION_TYPE, DATA
    46                              <2>   %xdefine INTERNAL_DATA_TO_CODE_RELOCATIONS INTERNAL_DATA_TO_CODE_RELOCATIONS, %%entry
    47                              <2>  %else
    48                              <2>   %xdefine INTERNAL_CODE_TO_CODE_RELOCATIONS INTERNAL_CODE_TO_CODE_RELOCATIONS, %%entry
    49                              <2>  %endif
    50                              <2> %endif
    51                              <2> 	eldstrictcheck
    52                              <2> 	%endmacro
    53                              <2> 
    54                              <2> 	%imacro internaldatarelocation 0-1.nolist -2
    55                              <2> %assign %%entry $ + _CURRENT_SECTION %+ FIXUP + %1
    56                              <2> %if ELDLINKER
    57                              <2>  %ifidni _CURRENT_SECTION_TYPE, DATA
    58                              <2>   %xdefine INTERNAL_LINKER_DATA_TO_DATA_RELOCATIONS INTERNAL_LINKER_DATA_TO_DATA_RELOCATIONS, %%entry
    59                              <2>  %else
    60                              <2>   %xdefine INTERNAL_LINKER_CODE_TO_DATA_RELOCATIONS INTERNAL_LINKER_CODE_TO_DATA_RELOCATIONS, %%entry
    61                              <2>  %endif
    62                              <2> %else
    63                              <2>  %ifidni _CURRENT_SECTION_TYPE, DATA
    64                              <2>   %xdefine INTERNAL_DATA_TO_DATA_RELOCATIONS INTERNAL_DATA_TO_DATA_RELOCATIONS, %%entry
    65                              <2>  %else
    66                              <2>   %xdefine INTERNAL_CODE_TO_DATA_RELOCATIONS INTERNAL_CODE_TO_DATA_RELOCATIONS, %%entry
    67                              <2>  %endif
    68                              <2> %endif
    69                              <2> 	eldstrictcheck
    70                              <2> 	%endmacro
    71                              <2> 
    72                              <2> ; dw INTERNAL_LINKER_CODE_TO_CODE_RELOCATIONS, 0
    73                              <2> ; dw INTERNAL_LINKER_CODE_TO_DATA_RELOCATIONS, 0
    74                              <2> ; dw INTERNAL_LINKER_DATA_TO_CODE_RELOCATIONS, -1
    75                              <2> ; dw INTERNAL_LINKER_DATA_TO_DATA_RELOCATIONS, -1
    76                              <2> ; dw INTERNAL_CODE_TO_CODE_RELOCATIONS, 0
    77                              <2> ; dw INTERNAL_CODE_TO_DATA_RELOCATIONS, 0
    78                              <2> ; dw INTERNAL_DATA_TO_CODE_RELOCATIONS, -1
    79                              <2> ; dw INTERNAL_DATA_TO_DATA_RELOCATIONS, -1
    80                              <2> 
    81                              <2> 
    82                              <2> %define LINK_DATA_RELOCATIONS ""
    83                              <2> %define LINK_LINKER_DATA_RELOCATIONS ""
    84                              <2> %define LINK_DATA_NAMES db ""
    85                              <2> %define LINK_DATA_DETECTION none, none
    86                              <2> 
    87                              <2> %define LINK_OTHER_DATA_RELOCATIONS ""
    88                              <2> %define LINK_OTHER_LINKER_DATA_RELOCATIONS ""
    89                              <2> %define LINK_OTHER_DATA_NAMES db ""
    90                              <2> %define LINK_OTHER_DATA_DETECTION none, none
    91                              <2> 
    92                              <2> %ifndef ELDOTHER
    93                              <2>  %assign ELDOTHER 0
    94                              <2> %endif
    95                              <2> %assign ELDOTHERLINK 0
    96                              <2> 
    97                              <2> 	%imacro otherlinkdatarelocation 1-3.nolist -2, required
    98                              <2> %if ELDOTHER
    99                              <2>  %assign ELDOTHERLINK 1
   100                              <2> %endif
   101                              <2> 	linkdatarelocation %1, %2, %3
   102                              <2> %assign ELDOTHERLINK 0
   103                              <2> 	%endmacro
   104                              <2> 
   105                              <2> 	%imacro linkdatarelocation 1-3.nolist -2, required
   106                              <2> %assign %%entry $ + _CURRENT_SECTION %+ FIXUP + %2
   107                              <2> %ifidni %3, required
   108                              <2>  %assign %%optional 0
   109                              <2> %elifidni %3, optional
   110                              <2>  %assign %%optional 100h
   111                              <2>  %if ELDDATA_OPTIONAL_STATUS == 0
   112                              <2>   %assign ELDDATA_OPTIONAL_STATUS 1
   113                              <2>  %elif ELDDATA_OPTIONAL_STATUS == 1
   114                              <2>  %else
   115                              <2>   %error Optional data link not allowed here
   116                              <2>  %endif
   117                              <2> %elifidni %3, PM required
   118                              <2>  %assign %%optional 300h
   119                              <2>  %assign ELDDATA_PMREQUIRED_STATUS 1
   120                              <2>  %if ELDDATA_OPTIONAL_STATUS == 0
   121                              <2>   %assign ELDDATA_OPTIONAL_STATUS 1
   122                              <2>  %elif ELDDATA_OPTIONAL_STATUS == 1
   123                              <2>  %else
   124                              <2>   %error Optional data link not allowed here
   125                              <2>  %endif
   126                              <2> %else
   127                              <2>  %fatal Unknown optional keyword
   128                              <2> %endif
   129                              <2> %ifidni _CURRENT_SECTION_TYPE, DATA
   130                              <2>  %assign %%DATASECTION 1
   131                              <2> %else
   132                              <2>  %assign %%DATASECTION 0
   133                              <2> %endif
   134                              <2> 	%if ELDOTHERLINK
   135                              <2> %if ELDLINKER
   136                              <2>  %xdefine LINK_OTHER_LINKER_DATA_RELOCATIONS LINK_OTHER_LINKER_DATA_RELOCATIONS, 1 + %%DATASECTION + %%optional, %%entry, %%name
   137                              <2> %else
   138                              <2>  %xdefine LINK_OTHER_DATA_RELOCATIONS LINK_OTHER_DATA_RELOCATIONS, 1 + %%DATASECTION + %%optional, %%entry, %%name
   139                              <2> %endif
   140                              <2> 	%else
   141                              <2> %if ELDLINKER
   142                              <2>  %xdefine LINK_LINKER_DATA_RELOCATIONS LINK_LINKER_DATA_RELOCATIONS, 1 + %%DATASECTION + %%optional, %%entry, %%name
   143                              <2> %else
   144                              <2>  %xdefine LINK_DATA_RELOCATIONS LINK_DATA_RELOCATIONS, 1 + %%DATASECTION + %%optional, %%entry, %%name
   145                              <2> %endif
   146                              <2> 	%endif
   147                              <2> %defstr %%string %1
   148                              <2> %strlen %%length %%string
   149                              <2> %if %%length > 64
   150                              <2>  %error Too long link name: %1
   151                              <2> %endif
   152                              <2> %define LINK_DATA_CHECK %1
   153                              <2> 	%if ELDOTHERLINK
   154                              <2> 	linkdata_detect LINK_OTHER_DATA_DETECTION
   155                              <2> %if LINK_DATA_NEW
   156                              <2>  %xdefine LINK_OTHER_DATA_DETECTION LINK_OTHER_DATA_DETECTION, %1, %%name
   157                              <2> 	hashdef HASH, %%string
   158                              <2>  %xdefine LINK_OTHER_DATA_NAMES 	LINK_OTHER_DATA_NAMES, %%name:, dw _HASH, {counted %%string}
   160                              <2> %else
   161                              <2>  %%name equ LINK_DATA_DUPLICATE
   162                              <2> %endif
   163                              <2> 	%else
   164                              <2> 	linkdata_detect LINK_DATA_DETECTION
   165                              <2> %if LINK_DATA_NEW
   166                              <2>  %xdefine LINK_DATA_DETECTION LINK_DATA_DETECTION, %1, %%name
   167                              <2> 	hashdef HASH, %%string
   168                              <2>  %xdefine LINK_DATA_NAMES 	LINK_DATA_NAMES, %%name:, dw _HASH, {counted %%string}
   170                              <2> %else
   171                              <2>  %%name equ LINK_DATA_DUPLICATE
   172                              <2> %endif
   173                              <2> 	%endif
   174                              <2> 	eldstrictcheck
   175                              <2> 	%endmacro
   176                              <2> 
   177                              <2> 	%imacro linkdata_detect 2-*.nolist
   178                              <2> %assign LINK_DATA_NEW 1
   179                              <2> %rep (%0 - 2) / 2
   180                              <2>  %rotate 2
   181                              <2>  %ifidni %1, LINK_DATA_CHECK
   182                              <2>   %assign LINK_DATA_NEW 0
   183                              <2>   %xdefine LINK_DATA_DUPLICATE %2
   184                              <2>   %exitrep
   185                              <2>  %endif
   186                              <2> %endrep
   187                              <2> 	%endmacro
   188                              <2> 
   189                              <2> 	%imacro link_data_dump_names 1-*.nolist
   190                              <2> %rep %0
   191                              <2> 	%1
   192                              <2>  %rotate 1
   193                              <2> %endrep
   194                              <2> 	%endmacro
   195                              <2> 
   196                              <2> ; dw LINK_LINKER_DATA_RELOCATIONS, 0, 0
   197                              <2> ; dw LINK_DATA_RELOCATIONS, 0, 0
   198                              <2> ; link_data_dump_names ELDCALL_CODE_NAMES
   199                              <2> 
   200                              <2> %endif
    21                              <1> 
    22                              <1> %assign ELDLINKER 0
    23                              <1> 
    24                              <1> [section relocatedzero nobits vstart=0]
    25                              <1> relocatedzero:
    26                              <1> __SECT__
    27                              <1> 
    28                              <1> 	numdef HOUDINI, 1
    29                              <1> 	numdef HOUDINI_CONDITIONAL, 1
    30                              <1> 
    31                              <1> %imacro houdini 0.nolist
    32                              <1> %if _HOUDINI
    33                              <1>  %if _HOUDINI_CONDITIONAL
    34                              <1> reloc	testopt [ss:relocateddata], 100h
    35                              <1> linkdatarelocation options7, -3
    36                              <1> 	jz %%skip
    37                              <1>  %endif
    38                              <1> reloc	testopt [ss:relocateddata], 100h
    39                              <1> linkdatarelocation internalflags6, -3
    40                              <1> 	jz %%skip
    41                              <1> 	int3
    42                              <1> %%skip:
    43                              <1> %endif
    44                              <1> %endmacro
    45                              <1> 
    46                              <1> %define ELDCALL_CODE_RELOCATIONS ""
    47                              <1> %define ELDCALL_LINKER_CODE_RELOCATIONS ""
    48                              <1> %define ELDCALL_CODE_RELOCATIONS_OPTIONAL ""
    49                              <1> %define ELDCALL_LINKER_CODE_RELOCATIONS_OPTIONAL ""
    50                              <1> %define ELDCALL_CODE_NAMES db ""
    51                              <1> %define ELDCALL_CODE_DETECTION none, none
    52                              <1> %assign ELDCALL_OPTIONAL_STATUS 0		; not any seen yet
    53                              <1> %assign ELDCALL_PMREQUIRED_STATUS 0		; not any seen yet
    54                              <1> 
    55                              <1> 	%imacro extcall 1-2.nolist required
    56                              <1> %ifidni _CURRENT_SECTION_TYPE, DATA
    57                              <1>  %error "ELD call cannot be used in ELD data block"
    58                              <1> %endif
    59                              <1> %assign %%entry $ + _CURRENT_SECTION %+ FIXUP
    60                              <1> %ifidni %2, required
    61                              <1>  %assign %%optional 0
    62                              <1> %elifidni %2, optional
    63                              <1>  %assign %%optional 100h
    64                              <1>  %if ELDCALL_OPTIONAL_STATUS == 0
    65                              <1>   %assign ELDCALL_OPTIONAL_STATUS 1
    66                              <1>  %elif ELDCALL_OPTIONAL_STATUS == 1
    67                              <1>  %else
    68                              <1>   %error Optional code link not allowed here
    69                              <1>  %endif
    70                              <1> %elifidni %2, PM required
    71                              <1>  %assign %%optional 300h
    72                              <1>  %assign ELDCALL_PMREQUIRED_STATUS 1
    73                              <1>  %if ELDCALL_OPTIONAL_STATUS == 0
    74                              <1>   %assign ELDCALL_OPTIONAL_STATUS 1
    75                              <1>  %elif ELDCALL_OPTIONAL_STATUS == 1
    76                              <1>  %else
    77                              <1>   %error Optional code link not allowed here
    78                              <1>  %endif
    79                              <1> %else
    80                              <1>  %fatal Unknown optional keyword
    81                              <1> %endif
    82                              <1> %if 0
    83                              <1> [warning -reloc-rel-word]
    84                              <1> 	call near relocatedzero
    85                              <1> [warning +reloc-rel-word]
    86                              <1> %else
    87                              <1> 	db 0E8h
    88                              <1> reloc	dw relocatedzero
    89                              <1> 	eldstrictcheck
    90                              <1> %endif
    91                              <1> 	jmp strict short %%skipparameter
    92                              <1> 	dw 0
    93                              <1> %%skipparameter:
    94                              <1> %if ELDLINKER
    95                              <1>  %xdefine ELDCALL_LINKER_CODE_RELOCATIONS ELDCALL_LINKER_CODE_RELOCATIONS, %%entry, %%name
    96                              <1>  %xdefine ELDCALL_LINKER_CODE_RELOCATIONS_OPTIONAL ELDCALL_LINKER_CODE_RELOCATIONS_OPTIONAL, 1 + %%optional, %%entry, %%name
    97                              <1> %else
    98                              <1>  %xdefine ELDCALL_CODE_RELOCATIONS ELDCALL_CODE_RELOCATIONS, %%entry, %%name
    99                              <1>  %xdefine ELDCALL_CODE_RELOCATIONS_OPTIONAL ELDCALL_CODE_RELOCATIONS_OPTIONAL, 1 + %%optional, %%entry, %%name
   100                              <1> %endif
   101                              <1> %defstr %%string %1
   102                              <1> %strlen %%length %%string
   103                              <1> %if %%length > 64
   104                              <1>  %error Too long link name: %1
   105                              <1> %endif
   106                              <1> %define ELDCALL_CODE_CHECK %1
   107                              <1> 	linkcode_detect ELDCALL_CODE_DETECTION
   108                              <1> %if ELDCALL_CODE_NEW
   109                              <1>  %xdefine ELDCALL_CODE_DETECTION ELDCALL_CODE_DETECTION, %1, %%name
   110                              <1> 	hashdef HASH, %%string
   111                              <1> %xdefine ELDCALL_CODE_NAMES 	ELDCALL_CODE_NAMES, %%name:, dw _HASH, {counted %%string}
   113                              <1> %else
   114                              <1>  %%name equ ELDCALL_CODE_DUPLICATE
   115                              <1> %endif
   116                              <1> 	%endmacro
   117                              <1> 
   118                              <1> 	%imacro linkcode_detect 2-*.nolist
   119                              <1> %assign ELDCALL_CODE_NEW 1
   120                              <1> %rep (%0 - 2) / 2
   121                              <1>  %rotate 2
   122                              <1>  %ifidni %1, ELDCALL_CODE_CHECK
   123                              <1>   %assign ELDCALL_CODE_NEW 0
   124                              <1>   %xdefine ELDCALL_CODE_DUPLICATE %2
   125                              <1>   %exitrep
   126                              <1>  %endif
   127                              <1> %endrep
   128                              <1> 	%endmacro
   129                              <1> 
   130                              <1> 
   131                              <1> %define ELDCALL_CALLCALL_LIST none
   132                              <1> 
   133                              <1> 	%imacro extcallcall 1.nolist
   134                              <1> 	call %1
   135                              <1> %xdefine ELDCALL_CALLCALL_LIST ELDCALL_CALLCALL_LIST, %1
   136                              <1> 	%endmacro
   137                              <1> 
   138                              <1> %assign ELDCALLCALL_DUMPED 0
   139                              <1> 
   140                              <1> 	%imacro eldcall_dump_callcall 1-*.nolist
   141                              <1> %define ELDCALL_CALLCALL_PROCESSED none
   142                              <1>  %rep %0 - 1
   143                              <1>   %rotate 1
   144                              <1>   %define ELDCALL_CHECK %1
   145                              <1> 	eldcall_callcall_detect ELDCALL_CALLCALL_PROCESSED
   146                              <1>   %if ELDCALL_NEW
   147                              <1>    %xdefine ELDCALL_CALLCALL_PROCESSED ELDCALL_CALLCALL_PROCESSED, %1
   148                              <1> 	align 8, nop
   149                              <1> %1:
   150                              <1> 	extcall %1
   151                              <1> 	retn
   152                              <1>   %endif
   153                              <1>  %endrep
   154                              <1> %unimacro extcallcall 1.nolist
   155                              <1> %assign ELDCALLCALL_DUMPED 1
   156                              <1> %define ELDCALL_CALLCALL_LIST none
   157                              <1> 	%endmacro
   158                              <1> 
   159                              <1> 	%imacro eldcall_callcall_detect 1-*.nolist
   160                              <1> %assign ELDCALL_NEW 1
   161                              <1> %rep %0 - 1
   162                              <1>  %rotate 1
   163                              <1>  %ifidni %1, ELDCALL_CHECK
   164                              <1>   %assign ELDCALL_NEW 0
   165                              <1>   %exitrep
   166                              <1>  %endif
   167                              <1> %endrep
   168                              <1> 	%endmacro
   169                              <1> 
   170                              <1> 	%imacro eldcall_dump_names 1-*.nolist
   171                              <1> %rep %0
   172                              <1> 	%1
   173                              <1>  %rotate 1
   174                              <1> %endrep
   175                              <1> 	%endmacro
   176                              <1> 
   177                              <1> ; eldcall_dump_callcall ELDCALL_CALLCALL_LIST
   178                              <1> ; if using optional code links:
   179                              <1> ;  dw ELDCALL_LINKER_CODE_RELOCATIONS_OPTIONAL, 0
   180                              <1> ;  dw ELDCALL_CODE_RELOCATIONS_OPTIONAL, 0
   181                              <1> ; if not using optional code links:
   182                              <1> ;  dw ELDCALL_LINKER_CODE_RELOCATIONS, 0, 0
   183                              <1> ;  dw ELDCALL_CODE_RELOCATIONS, 0, 0
   184                              <1> ; eldcall_dump_names ELDCALL_CODE_NAMES
   185                              <1> 
   186                              <1> %endif
    10                                  %include "elddata.mac"
     1                              <1> %if 0
     2                              <1> 
     3                              <1> Extensions for lDebug data relocation macros
     4                              <1> 
     5                              <1> Copyright (C) 2008-2024 E. C. Masloch
     6                              <1> 
     7                              <1> Usage of the works is permitted provided that this
     8                              <1> instrument is retained with the works, so that any entity
     9                              <1> that uses the works is notified of this instrument.
    10                              <1> 
    11                              <1> DISCLAIMER: THE WORKS ARE WITHOUT WARRANTY.
    12                              <1> 
    13                              <1> %endif
    14                              <1> 
    15                              <1> %ifndef ELDDATA_MAC
    16                              <1> %define ELDDATA_MAC 1
    17                              <1> 
    18                              <1> %include "lmacros3.mac"
    19                              <1> %include "nasmhash.mac"
    20                              <1> %include "eldcheck.mac"
    21                              <1> 
    22                              <1> 
    23                              <1> %assign ELDLINKER 0
    24                              <1> 
    25                              <1> %define INTERNAL_CODE_TO_CODE_RELOCATIONS ""
    26                              <1> %define INTERNAL_CODE_TO_DATA_RELOCATIONS ""
    27                              <1> %define INTERNAL_DATA_TO_CODE_RELOCATIONS ""
    28                              <1> %define INTERNAL_DATA_TO_DATA_RELOCATIONS ""
    29                              <1> %define INTERNAL_LINKER_CODE_TO_CODE_RELOCATIONS ""
    30                              <1> %define INTERNAL_LINKER_CODE_TO_DATA_RELOCATIONS ""
    31                              <1> %define INTERNAL_LINKER_DATA_TO_CODE_RELOCATIONS ""
    32                              <1> %define INTERNAL_LINKER_DATA_TO_DATA_RELOCATIONS ""
    33                              <1> %assign ELDDATA_OPTIONAL_STATUS 0		; not any seen yet
    34                              <1> %assign ELDDATA_PMREQUIRED_STATUS 0		; not any seen yet
    35                              <1> 
    36                              <1> 	%imacro internalcoderelocation 0-1.nolist -2
    37                              <1> %assign %%entry $ + _CURRENT_SECTION %+ FIXUP + %1
    38                              <1> %if ELDLINKER
    39                              <1>  %ifidni _CURRENT_SECTION_TYPE, DATA
    40                              <1>   %xdefine INTERNAL_LINKER_DATA_TO_CODE_RELOCATIONS INTERNAL_LINKER_DATA_TO_CODE_RELOCATIONS, %%entry
    41                              <1>  %else
    42                              <1>   %xdefine INTERNAL_LINKER_CODE_TO_CODE_RELOCATIONS INTERNAL_LINKER_CODE_TO_CODE_RELOCATIONS, %%entry
    43                              <1>  %endif
    44                              <1> %else
    45                              <1>  %ifidni _CURRENT_SECTION_TYPE, DATA
    46                              <1>   %xdefine INTERNAL_DATA_TO_CODE_RELOCATIONS INTERNAL_DATA_TO_CODE_RELOCATIONS, %%entry
    47                              <1>  %else
    48                              <1>   %xdefine INTERNAL_CODE_TO_CODE_RELOCATIONS INTERNAL_CODE_TO_CODE_RELOCATIONS, %%entry
    49                              <1>  %endif
    50                              <1> %endif
    51                              <1> 	eldstrictcheck
    52                              <1> 	%endmacro
    53                              <1> 
    54                              <1> 	%imacro internaldatarelocation 0-1.nolist -2
    55                              <1> %assign %%entry $ + _CURRENT_SECTION %+ FIXUP + %1
    56                              <1> %if ELDLINKER
    57                              <1>  %ifidni _CURRENT_SECTION_TYPE, DATA
    58                              <1>   %xdefine INTERNAL_LINKER_DATA_TO_DATA_RELOCATIONS INTERNAL_LINKER_DATA_TO_DATA_RELOCATIONS, %%entry
    59                              <1>  %else
    60                              <1>   %xdefine INTERNAL_LINKER_CODE_TO_DATA_RELOCATIONS INTERNAL_LINKER_CODE_TO_DATA_RELOCATIONS, %%entry
    61                              <1>  %endif
    62                              <1> %else
    63                              <1>  %ifidni _CURRENT_SECTION_TYPE, DATA
    64                              <1>   %xdefine INTERNAL_DATA_TO_DATA_RELOCATIONS INTERNAL_DATA_TO_DATA_RELOCATIONS, %%entry
    65                              <1>  %else
    66                              <1>   %xdefine INTERNAL_CODE_TO_DATA_RELOCATIONS INTERNAL_CODE_TO_DATA_RELOCATIONS, %%entry
    67                              <1>  %endif
    68                              <1> %endif
    69                              <1> 	eldstrictcheck
    70                              <1> 	%endmacro
    71                              <1> 
    72                              <1> ; dw INTERNAL_LINKER_CODE_TO_CODE_RELOCATIONS, 0
    73                              <1> ; dw INTERNAL_LINKER_CODE_TO_DATA_RELOCATIONS, 0
    74                              <1> ; dw INTERNAL_LINKER_DATA_TO_CODE_RELOCATIONS, -1
    75                              <1> ; dw INTERNAL_LINKER_DATA_TO_DATA_RELOCATIONS, -1
    76                              <1> ; dw INTERNAL_CODE_TO_CODE_RELOCATIONS, 0
    77                              <1> ; dw INTERNAL_CODE_TO_DATA_RELOCATIONS, 0
    78                              <1> ; dw INTERNAL_DATA_TO_CODE_RELOCATIONS, -1
    79                              <1> ; dw INTERNAL_DATA_TO_DATA_RELOCATIONS, -1
    80                              <1> 
    81                              <1> 
    82                              <1> %define LINK_DATA_RELOCATIONS ""
    83                              <1> %define LINK_LINKER_DATA_RELOCATIONS ""
    84                              <1> %define LINK_DATA_NAMES db ""
    85                              <1> %define LINK_DATA_DETECTION none, none
    86                              <1> 
    87                              <1> %define LINK_OTHER_DATA_RELOCATIONS ""
    88                              <1> %define LINK_OTHER_LINKER_DATA_RELOCATIONS ""
    89                              <1> %define LINK_OTHER_DATA_NAMES db ""
    90                              <1> %define LINK_OTHER_DATA_DETECTION none, none
    91                              <1> 
    92                              <1> %ifndef ELDOTHER
    93                              <1>  %assign ELDOTHER 0
    94                              <1> %endif
    95                              <1> %assign ELDOTHERLINK 0
    96                              <1> 
    97                              <1> 	%imacro otherlinkdatarelocation 1-3.nolist -2, required
    98                              <1> %if ELDOTHER
    99                              <1>  %assign ELDOTHERLINK 1
   100                              <1> %endif
   101                              <1> 	linkdatarelocation %1, %2, %3
   102                              <1> %assign ELDOTHERLINK 0
   103                              <1> 	%endmacro
   104                              <1> 
   105                              <1> 	%imacro linkdatarelocation 1-3.nolist -2, required
   106                              <1> %assign %%entry $ + _CURRENT_SECTION %+ FIXUP + %2
   107                              <1> %ifidni %3, required
   108                              <1>  %assign %%optional 0
   109                              <1> %elifidni %3, optional
   110                              <1>  %assign %%optional 100h
   111                              <1>  %if ELDDATA_OPTIONAL_STATUS == 0
   112                              <1>   %assign ELDDATA_OPTIONAL_STATUS 1
   113                              <1>  %elif ELDDATA_OPTIONAL_STATUS == 1
   114                              <1>  %else
   115                              <1>   %error Optional data link not allowed here
   116                              <1>  %endif
   117                              <1> %elifidni %3, PM required
   118                              <1>  %assign %%optional 300h
   119                              <1>  %assign ELDDATA_PMREQUIRED_STATUS 1
   120                              <1>  %if ELDDATA_OPTIONAL_STATUS == 0
   121                              <1>   %assign ELDDATA_OPTIONAL_STATUS 1
   122                              <1>  %elif ELDDATA_OPTIONAL_STATUS == 1
   123                              <1>  %else
   124                              <1>   %error Optional data link not allowed here
   125                              <1>  %endif
   126                              <1> %else
   127                              <1>  %fatal Unknown optional keyword
   128                              <1> %endif
   129                              <1> %ifidni _CURRENT_SECTION_TYPE, DATA
   130                              <1>  %assign %%DATASECTION 1
   131                              <1> %else
   132                              <1>  %assign %%DATASECTION 0
   133                              <1> %endif
   134                              <1> 	%if ELDOTHERLINK
   135                              <1> %if ELDLINKER
   136                              <1>  %xdefine LINK_OTHER_LINKER_DATA_RELOCATIONS LINK_OTHER_LINKER_DATA_RELOCATIONS, 1 + %%DATASECTION + %%optional, %%entry, %%name
   137                              <1> %else
   138                              <1>  %xdefine LINK_OTHER_DATA_RELOCATIONS LINK_OTHER_DATA_RELOCATIONS, 1 + %%DATASECTION + %%optional, %%entry, %%name
   139                              <1> %endif
   140                              <1> 	%else
   141                              <1> %if ELDLINKER
   142                              <1>  %xdefine LINK_LINKER_DATA_RELOCATIONS LINK_LINKER_DATA_RELOCATIONS, 1 + %%DATASECTION + %%optional, %%entry, %%name
   143                              <1> %else
   144                              <1>  %xdefine LINK_DATA_RELOCATIONS LINK_DATA_RELOCATIONS, 1 + %%DATASECTION + %%optional, %%entry, %%name
   145                              <1> %endif
   146                              <1> 	%endif
   147                              <1> %defstr %%string %1
   148                              <1> %strlen %%length %%string
   149                              <1> %if %%length > 64
   150                              <1>  %error Too long link name: %1
   151                              <1> %endif
   152                              <1> %define LINK_DATA_CHECK %1
   153                              <1> 	%if ELDOTHERLINK
   154                              <1> 	linkdata_detect LINK_OTHER_DATA_DETECTION
   155                              <1> %if LINK_DATA_NEW
   156                              <1>  %xdefine LINK_OTHER_DATA_DETECTION LINK_OTHER_DATA_DETECTION, %1, %%name
   157                              <1> 	hashdef HASH, %%string
   158                              <1>  %xdefine LINK_OTHER_DATA_NAMES 	LINK_OTHER_DATA_NAMES, %%name:, dw _HASH, {counted %%string}
   160                              <1> %else
   161                              <1>  %%name equ LINK_DATA_DUPLICATE
   162                              <1> %endif
   163                              <1> 	%else
   164                              <1> 	linkdata_detect LINK_DATA_DETECTION
   165                              <1> %if LINK_DATA_NEW
   166                              <1>  %xdefine LINK_DATA_DETECTION LINK_DATA_DETECTION, %1, %%name
   167                              <1> 	hashdef HASH, %%string
   168                              <1>  %xdefine LINK_DATA_NAMES 	LINK_DATA_NAMES, %%name:, dw _HASH, {counted %%string}
   170                              <1> %else
   171                              <1>  %%name equ LINK_DATA_DUPLICATE
   172                              <1> %endif
   173                              <1> 	%endif
   174                              <1> 	eldstrictcheck
   175                              <1> 	%endmacro
   176                              <1> 
   177                              <1> 	%imacro linkdata_detect 2-*.nolist
   178                              <1> %assign LINK_DATA_NEW 1
   179                              <1> %rep (%0 - 2) / 2
   180                              <1>  %rotate 2
   181                              <1>  %ifidni %1, LINK_DATA_CHECK
   182                              <1>   %assign LINK_DATA_NEW 0
   183                              <1>   %xdefine LINK_DATA_DUPLICATE %2
   184                              <1>   %exitrep
   185                              <1>  %endif
   186                              <1> %endrep
   187                              <1> 	%endmacro
   188                              <1> 
   189                              <1> 	%imacro link_data_dump_names 1-*.nolist
   190                              <1> %rep %0
   191                              <1> 	%1
   192                              <1>  %rotate 1
   193                              <1> %endrep
   194                              <1> 	%endmacro
   195                              <1> 
   196                              <1> ; dw LINK_LINKER_DATA_RELOCATIONS, 0, 0
   197                              <1> ; dw LINK_DATA_RELOCATIONS, 0, 0
   198                              <1> ; link_data_dump_names ELDCALL_CODE_NAMES
   199                              <1> 
   200                              <1> %endif
    11                                  
    12                                  	cpu 8086
    13                                  
    14                                  	addsection RELOCATEDDATA, nobits vstart=_ELD_RELOC_VSTART
    15                                  relocateddata:
    16                                  
    17                                  	addsection HEADER, start=0
    18                                  
    19                                  	istruc ELD_HEADERX
    20                                  at eldhxHeader
    21                                  		; ELD executable header
    22                                  	istruc ELD_HEADER
    23 00000000 454C4431                at eldhSignature,	db "ELD1"
    24 00000004 000000                  			db 0,0,0
    25 00000007 1A                      			db 26
    26 00000008 70000000                at eldhCodeOffset,	dd CODEOFFSET
    27 0000000C 800B                    at eldhCodeImageLength,	dw code_size
    28 0000000E 0000                    at eldhCodeAllocLength,	dw 0
    29 00000010 F00B0000                at eldhDataOffset,	dd DATAOFFSET
    30 00000014 1003                    at eldhDataImageLength,	dw data_size
    31 00000016 0000                    at eldhDataAllocLength,	dw total_data_size - data_size
    32 00000018 FE03                    at eldhCodeEntrypoint,	dw linker - code
    33                                  at eldhReserved
    34 0000001A 00<rep 4h>2800          at eldhExtensionSize,	dw header_extension_end - $$
    35                                  	iend
    36 00000020 [30000000]              at eldhxDescriptionOffset,	dd description
    37 00000024 3D0D0000                at eldhxHelpOffset,		dd DATAOFFSET + msg.help - datastart
    38                                  PUT_ELDHX_DATETIME_OFFSET
    39                                  header_extension_end:
    40 00000028 00<rep 8h>              	iend
    41                                  
    42 00000030 507574207365706172-     description:		asciz "Put separators in disassembly on control flow end."
    42 00000039 61746F727320696E20-
    42 00000042 646973617373656D62-
    42 0000004B 6C79206F6E20636F6E-
    42 00000054 74726F6C20666C6F77-
    42 0000005D 20656E642E00       
    43                                  
    44                                  
    45 00000063 00<rep Dh>              	align 16, db 0
    46                                  
    47                                  CODEOFFSET equ $ - $$
    48                                  	addsection CODE, follows=HEADER vstart=_ELD_CODE_VSTART
    49                                  %define CODEFIXUP - code + 0
    50                                  code:
    51                                  		; ELD instance header
    52                                  	istruc ELD_INSTANCE
    53                                  at eldiStartCode
    54 00000000 00<rep 2h>              at eldiEndCode
    55 00000002 00<rep 2h>              at eldiStartData
    56 00000004 00<rep 2h>              at eldiEndData
    57 00000006 00<rep 2h>55534550-     at eldiIdentifier,	fill 8, 32, db "USEPARAT"
    57 0000000C 41524154           
    58 00000010 00<rep 2h>75736570-     at eldiListing,		asciz _ELD_LISTING
    58 00000016 617261742E6C737400 
    59 0000001F 00                      	iend
    60                                  
    61                                  
    62                                  command:
    63 00000020 EB08                    	jmp strict short .entry
    64                                  .chain:
    65 00000022 E8[0000]EB020000        	extcall cmd3_not_ext, required	; must NOT be extcallcall
    66 00000029 90                      	times 10 - ($ - command) nop
    67                                  .entry:
    68 0000002A 56                      	push si
    69 0000002B 3C2D                    	cmp al, '-'
    70 0000002D 7503                    	jne @F
    71 0000002F E8BE02                  	extcallcall skipcomma
    72                                  @@:
    73 00000032 4E                      	dec si
    74                                  
    75 00000033 BA[2500]                	mov dx, msg.useparat
    76                                  internaldatarelocation
    77 00000036 E8BF02                  	extcallcall isstring?
    78 00000039 7405                    	je .ours
    79 0000003B 5E                      	pop si
    80 0000003C 4E                      	dec si
    81 0000003D AC                      	lodsb
    82 0000003E EBE2                    	jmp .chain
    83                                  
    84                                  .ours:
    85 00000040 58                      	pop ax
    86 00000041 E8AC02                  	extcallcall skipcomma
    87 00000044 4E                      	dec si
    88 00000045 C706[0000][0000]        reloc2	mov word [relocateddata], relocateddata
    89                                  linkdatarelocation lastcmd, -4
    90                                  linkdatarelocation dmycmd
    91 0000004B BA[0000]                	mov dx, relocateddata
    92                                  linkdatarelocation msg.uninstall
    93 0000004E E8A702                  	extcallcall isstring?
    94 00000051 7503E9E901              	je uninstall
    95 00000056 BA[6600]                	mov dx, msg.width
    96                                  internaldatarelocation
    97 00000059 E89C02                  	extcallcall isstring?
    98 0000005C 7503E9C801              	je setwidth
    99 00000061 AC                      	lodsb
   100 00000062 E89B02                  	extcallcall chkeol
   101 00000065 E8A002                  	extcallcall cmd3
   102                                  
   103                                  
   104                                  puts_handler:
   105                                  .:
   106 00000068 EB08                    	jmp strict short .entry
   107                                  .chain:
   108 0000006A E8[0000]EB020000        	extcall puts_ext_done, required	; must NOT be extcallcall
   109 00000071 90                      	times 10 - ($ - .) nop
   110                                  .entry:
   111                                  
   112                                  		; es:dx -> message
   113                                  		; ax = length
   114 00000072 56                      	push si
   115 00000073 57                      	push di
   116 00000074 50                      	push ax
   117 00000075 06                      	push es
   118 00000076 52                      	push dx
   119 00000077 1E                      	push ds
   120 00000078 06                      	 push es
   121 00000079 1F                      	 pop ds
   122                                  
   123 0000007A 368A0E[2300]            	mov cl, byte [ss:isregdump]
   124                                  internaldatarelocation
   125 0000007F 36880E[2400]            	mov byte [ss:wasregdump], cl
   126                                  internaldatarelocation
   127 00000084 36C606[2300]00          	mov byte [ss:isregdump], 0
   128                                  internaldatarelocation -3
   129                                  
   130 0000008A 89D6                    	mov si, dx
   131 0000008C 89C1                    	mov cx, ax
   132 0000008E 41                      	inc cx
   133                                  
   134 0000008F 83F803                  	cmp ax, 3
   135 00000092 7303E98201              	jb .notours
   136                                  
   137 00000097 807C023D                	cmp byte [si + 2], '='
   138 0000009B 7515                    	jne @F
   139 0000009D 813C4453                	cmp word [si], "DS"
   140 000000A1 7406                    	je .regdump
   141 000000A3 813C4950                	cmp word [si], "IP"
   142 000000A7 7509                    	jne @F
   143                                  .regdump:
   144 000000A9 36C606[2300]FF          	mov byte [ss:isregdump], 0FFh
   145                                  internaldatarelocation -3
   146 000000AF E96701                  	jmp .notours
   147                                  
   148                                  @@:
   149 000000B2 83F812                  	cmp ax, 4 + 1 + 4 + 1 + 8
   150 000000B5 7303E95F01              	jb .notours
   151                                  
   152                                  %imacro looplodsb 0
   153                                  	loop %%skip
   154                                  	jmp .notours
   155                                  %%skip:
   156                                  	lodsb
   157                                  %endmacro
   158                                  
   159 000000BA BA0400                  	mov dx, 4
   160                                  @@:
   161                                  	looplodsb
   153 000000BD E203                <1>  loop %%skip
   154 000000BF E95701              <1>  jmp .notours
   155                              <1> %%skip:
   156 000000C2 AC                  <1>  lodsb
   162 000000C3 E84A02                  	extcallcall getnyb
   163 000000C6 7303E94E01              	jc .notours
   164 000000CB 4A                      	dec dx
   165 000000CC 75EF                    	jnz @B
   166                                  	looplodsb
   153 000000CE E203                <1>  loop %%skip
   154 000000D0 E94601              <1>  jmp .notours
   155                              <1> %%skip:
   156 000000D3 AC                  <1>  lodsb
   167 000000D4 3C3A                    	cmp al, ':'
   168 000000D6 7403E93E01              	jne .notours
   169                                  
   170 000000DB B204                    	mov dl, 4
   171                                  @@:
   172                                  	looplodsb
   153 000000DD E203                <1>  loop %%skip
   154 000000DF E93701              <1>  jmp .notours
   155                              <1> %%skip:
   156 000000E2 AC                  <1>  lodsb
   173 000000E3 E82A02                  	extcallcall getnyb
   174 000000E6 7303E92E01              	jc .notours
   175 000000EB 4A                      	dec dx
   176 000000EC 75EF                    	jnz @B
   177                                  
   178 000000EE B204                    	mov dl, 4
   179                                  @@:
   180                                  	looplodsb
   153 000000F0 E203                <1>  loop %%skip
   154 000000F2 E92401              <1>  jmp .notours
   155                              <1> %%skip:
   156 000000F5 AC                  <1>  lodsb
   181 000000F6 E81702                  	extcallcall getnyb
   182 000000F9 7209                    	jc @F
   183 000000FB 4A                      	dec dx
   184 000000FC 75F2                    	jnz @B
   185                                  
   186                                  	looplodsb
   153 000000FE E203                <1>  loop %%skip
   154 00000100 E91601              <1>  jmp .notours
   155                              <1> %%skip:
   156 00000103 AC                  <1>  lodsb
   187                                  @@:
   188 00000104 3C20                    	cmp al, 32
   189 00000106 7403E90E01              	jne .notours
   190                                  @@:
   191                                  	looplodsb
   153 0000010B E203                <1>  loop %%skip
   154 0000010D E90901              <1>  jmp .notours
   155                              <1> %%skip:
   156 00000110 AC                  <1>  lodsb
   192 00000111 3C20                    	cmp al, 32
   193 00000113 74F6                    	je @B
   194 00000115 E8F801                  	extcallcall getnyb
   195 00000118 7303E9FC00              	jc .notours
   196                                  
   197 0000011D 817CFF4542              	cmp word [si - 1], "EB"
   198 00000122 7503E9F200              	je .notours
   199                                  @@:
   200                                  	looplodsb
   153 00000127 E203                <1>  loop %%skip
   154 00000129 E9ED00              <1>  jmp .notours
   155                              <1> %%skip:
   156 0000012C AC                  <1>  lodsb
   201 0000012D E8E001                  	extcallcall getnyb
   202 00000130 73F5                    	jnc @B
   203 00000132 3C20                    	cmp al, 32
   204 00000134 7403E9E000              	jne .notours
   205                                  
   206                                  @@:
   207                                  	looplodsb
   153 00000139 E203                <1>  loop %%skip
   154 0000013B E9DB00              <1>  jmp .notours
   155                              <1> %%skip:
   156 0000013E AC                  <1>  lodsb
   208 0000013F 3C20                    	cmp al, 32
   209 00000141 74F6                    	je @B
   210                                  
   211 00000143 4E                      	dec si
   212                                  
   213 00000144 BA[7F00]                	mov dx, msg.int
   214                                  internaldatarelocation
   215 00000147 16                      	 push ss
   216 00000148 07                      	 pop es
   217 00000149 E8AC01                  	extcallcall isstring?
   218 0000014C 7539                    	jne @FF
   219 0000014E E8C701                  	extcallcall skipwhite
   220 00000151 4E                      	dec si
   221                                  
   222 00000152 BA[8300]                	mov dx, msg.20
   223                                  internaldatarelocation
   224 00000155 E8A001                  	extcallcall isstring?
   225 00000158 7503E9A700              	je .terminate
   226                                  
   227 0000015D 36D006[2400]            	rol byte [ss:wasregdump], 1
   228                                  internaldatarelocation
   229 00000162 730B                    	jnc @F
   230                                  
   231 00000164 36803E[0100]4C          	cmp byte [ss:relocateddata + 1], 4Ch
   232                                  linkdatarelocation reg_eax, -3
   233 0000016A 740D                    	je .checkint21
   234 0000016C E9AA00                  	jmp .notours
   235                                  
   236                                  @@:
   237 0000016F 36D006[2200]            	rol byte [ss:mov_ah_4Ch], 1
   238                                  internaldatarelocation
   239 00000174 7203E9A000              	jnc .notours
   240                                  
   241                                  .checkint21:
   242 00000179 BA[8600]                	mov dx, msg.21
   243                                  internaldatarelocation
   244 0000017C E87901                  	extcallcall isstring?
   245 0000017F 7503E98000              	je .terminate
   246 00000184 E99200                  	jmp .notours
   247                                  
   248                                  @@:
   249                                  
   250 00000187 BF[1400]                	mov di, ah_4Ch_table - 4
   251                                  internaldatarelocation
   252 0000018A A8                      	db __TEST_IMM8			; skip pop
   253                                  @@:
   254 0000018B 5E                      	pop si
   255 0000018C 56                      	push si
   256 0000018D 8D7D04                  	lea di, [di + 4]
   257 00000190 368B15                  	mov dx, word [ss:di]
   258 00000193 85D2                    	test dx, dx
   259 00000195 742C                    	jz .not_ah_4Ch
   260 00000197 16                      	 push ss
   261 00000198 07                      	 pop es
   262 00000199 E85C01                  	extcallcall isstring?
   263 0000019C 75ED                    	jne @B
   264 0000019E E87701                  	extcallcall skipwhite
   265 000001A1 4E                      	dec si
   266 000001A2 368B5502                	mov dx, word [ss:di + 2]
   267 000001A6 E84F01                  	extcallcall isstring?
   268 000001A9 75E0                    	jne @B
   269 000001AB AC                      	lodsb
   270 000001AC 3C2C                    	cmp al, ','
   271 000001AE 7513                    	jne .not_ah_4Ch
   272 000001B0 E86D01                  	extcallcall skipcomm0
   273 000001B3 817CFF3443              	cmp word [si - 1], "4C"
   274 000001B8 75D1                    	jne @B
   275                                  
   276 000001BA 58                      	pop ax				; discard si
   277 000001BB 36C606[2200]FF          	mov byte [ss:mov_ah_4Ch], 0FFh
   278                                  internaldatarelocation -3
   279 000001C1 EB5C                    	jmp .notours_ah_4Ch
   280                                  
   281                                  
   282                                  .not_ah_4Ch:
   283 000001C3 5E                      	pop si
   284 000001C4 BF[0C00]                	mov di, table
   285                                  internaldatarelocation
   286                                  @@:
   287 000001C7 368B15                  	mov dx, word [ss:di]
   288 000001CA 85D2                    	test dx, dx
   289 000001CC 744B                    	jz .notours
   290 000001CE 16                      	 push ss
   291 000001CF 07                      	 pop es
   292 000001D0 E82501                  	extcallcall isstring?
   293 000001D3 8D7D02                  	lea di, [di + 2]
   294 000001D6 75EF                    	jne @B
   295                                  
   296 000001D8 1F                      	pop ds
   297 000001D9 5A                      	pop dx
   298 000001DA 07                      	pop es
   299 000001DB 58                      	pop ax
   300 000001DC 5F                      	pop di
   301 000001DD 5E                      	pop si
   302                                  
   303 000001DE B9[6A00]                	mov cx, .chain			; -> our chaining entry
   304                                  internalcoderelocation
   305 000001E1 F8                      	clc
   306 000001E2 E84301                  	extcallcall puts_ext_next	; call subsequent puts handlers
   307                                  
   308 000001E5 06                      	push es
   309 000001E6 16                      	 push ss
   310 000001E7 07                      	 pop es
   311 000001E8 BA[E300]                	mov dx, msg.separator + 80	; es:dx -> message
   312                                  internaldatarelocation
   313                                  @@:
   314 000001EB 36A1[1600]              	mov ax, word [ss:width]
   315                                  internaldatarelocation
   316 000001EF 29C2                    	sub dx, ax			; -> message to display
   317 000001F1 83C002                  	add ax, msg.separator_linebreak_size
   318                                  					; ax = length
   319 000001F4 B9[6A00]                	mov cx, .chain			; -> our chaining entry
   320                                  internalcoderelocation
   321 000001F7 F8                      	clc
   322 000001F8 E82D01                  	extcallcall puts_ext_next	; call subsequent puts handlers
   323 000001FB 07                      	pop es
   324                                  
   325 000001FC F9                      	stc
   326 000001FD E8[0000]EB020000        	extcall puts_ext_done, required
   327                                  					; directly jump back to debugger, CY
   328                                  
   329                                  .terminate:
   330 00000204 1F                      	pop ds
   331 00000205 5A                      	pop dx
   332 00000206 07                      	pop es
   333 00000207 58                      	pop ax
   334 00000208 5F                      	pop di
   335 00000209 5E                      	pop si
   336                                  
   337 0000020A B9[6A00]                	mov cx, .chain			; -> our chaining entry
   338                                  internalcoderelocation
   339 0000020D F8                      	clc
   340 0000020E E81701                  	extcallcall puts_ext_next	; call subsequent puts handlers
   341                                  
   342 00000211 06                      	push es
   343 00000212 16                      	 push ss
   344 00000213 07                      	 pop es
   345 00000214 BA[3501]                	mov dx, msg.separator_terminate + 80	; es:dx -> message
   346                                  internaldatarelocation
   347 00000217 EBD2                    	jmp @B
   348                                  
   349                                  
   350                                  .notours:
   351 00000219 36C606[2200]00          	mov byte [ss:mov_ah_4Ch], 0
   352                                  internaldatarelocation -3
   353                                  .notours_ah_4Ch:
   354                                  
   355 0000021F 1F                      	pop ds
   356 00000220 5A                      	pop dx
   357 00000221 07                      	pop es
   358 00000222 58                      	pop ax
   359 00000223 5F                      	pop di
   360 00000224 5E                      	pop si
   361                                  
   362 00000225 F8                      	clc
   363 00000226 E941FE                  	jmp .chain			; chain if to display -->
   364                                  
   365                                  
   366                                  setwidth:
   367 00000229 AC                      	lodsb
   368 0000022A E80301                  	extcallcall getbyte
   369 0000022D E8D000                  	extcallcall chkeol
   370 00000230 80FA50                  	cmp dl, 80
   371 00000233 7603                    	jbe @F
   372 00000235 E80001                  	extcallcall error
   373                                  
   374                                  @@:
   375 00000238 8816[1600]              	mov byte [width], dl
   376                                  internaldatarelocation
   377 0000023C E8C900                  	extcallcall cmd3
   378                                  
   379                                  
   380                                  uninstall:
   381 0000023F AC                      	lodsb
   382 00000240 E8BD00                  	extcallcall chkeol
   383                                  
   384 00000243 E89500                  	call get_es_ext
   385                                  
   386 00000246 06                      	push es
   387 00000247 1F                      	pop ds
   388                                  
   389 00000248 BE[0000]                	mov si, hooktable
   390                                  internaldatarelocation
   391                                  	lframe
   392 0000024B 5589E5                  	lenter
   393                                  	lvar word, table
   394 0000024E 56                      	 push si
   395                                  
   396                                  .loop_table:
   397 0000024F 36D04404                	rol byte [ss:si + htInstalled], 1
   398 00000253 735C                    	jnc .next_table
   399 00000255 31DB                    	xor bx, bx		; = 0 (no prior, modify handler)
   400 00000257 368B3C                  	mov di, word [ss:si + htEntry]	; di -> us
   401 0000025A 368B7402                	mov si, word [ss:si + htHandler]; -> handler
   402 0000025E 368B34                  	mov si, word [ss:si]	; si -> first
   403 00000261 85F6                    	test si, si		; none installed ?
   404 00000263 746B                    	jz .error		; error -->
   405                                  
   406                                  .loop:
   407 00000265 39F7                    	cmp di, si		; found ?
   408 00000267 740D                    	je .bx			; yes, use bx -->
   409 00000269 89F3                    	mov bx, si		; bx -> prior handler
   410 0000026B AD                      	lodsw			; skip entrypoint jmp strict short
   411 0000026C AC                      	lodsb			; get first byte of chainer
   412 0000026D 3CE9                    	cmp al, 0E9h		; expecting jmp near ?
   413 0000026F 755F                    	jne .error		; no, error -->
   414 00000271 AD                      	lodsw			; get rel16 displacement
   415 00000272 01C6                    	add si, ax		; -> next handler
   416 00000274 EBEF                    	jmp .loop
   417                                  
   418                                  .bx:
   419 00000276 85DB                    	test bx, bx		; any prior ?
   420 00000278 751F                    	jnz .bxnz		; yes -->
   421 0000027A AF                      	scasw			; skip entrypoint jmp strict short
   422 0000027B 803DE8                  	cmp byte [di], 0E8h	; is it a call to cmd3_not_ext ?
   423 0000027E 750C                    	jne @F			; no -->
   424                                  				; yes, reset ext_command_handler to zero
   425                                  .setbx:
   426 00000280 8B76FE                  	mov si, word [bp + ?table]
   427 00000283 368B7402                	mov si, word [ss:si + htHandler]; -> handler
   428 00000287 36891C                  	mov word [ss:si], bx
   429 0000028A EB1E                    	jmp .done
   430                                  
   431                                  @@:
   432 0000028C 803DE9                  	cmp byte [di], 0E9h	; validate
   433 0000028F 753F                    	jne .error		; failure -->
   434 00000291 47                      	inc di			; -> rel16 displacement
   435 00000292 8B1D                    	mov bx, word [di]	; get displacement
   436 00000294 AF                      	scasw			; -> after jmp near
   437 00000295 01FB                    	add bx, di		; -> next handler
   438 00000297 EBE7                    	jmp .setbx		; set ext_command_handler to next
   439                                  
   440                                  .bxnz:
   441 00000299 89DE                    	mov si, bx		; -> prior handler with us as downlink
   442 0000029B 87FE                    	xchg di, si		; si -> ours, di -> prior
   443 0000029D A7                      	cmpsw			; skip entrypoint jmp strict short
   444 0000029E A4                      	movsb			; copy 0E8h/0E9h
   445 0000029F AD                      	lodsw			; ax = near rel16 displacement
   446 000002A0 01F0                    	add ax, si		; add in our base (= absolute offset)
   447 000002A2 29F8                    	sub ax, di
   448 000002A4 48                      	dec ax
   449 000002A5 48                      	dec ax			; subtract new base (= relative displacement)
   450 000002A6 AB                      	stosw			; store new rel16 displacement
   451 000002A7 A5                      	movsw			; jmp strict short
   452 000002A8 A5                      	movsw			; linkcall target
   453 000002A9 A4                      	movsb			; trailer
   454                                  .done:
   455 000002AA 8B76FE                  	mov si, word [bp + ?table]
   456 000002AD 36F65404                	not byte [ss:si + htInstalled]
   457                                  
   458                                  .next_table:
   459 000002B1 83C606                  	add si, HOOKTABLE_size
   460 000002B4 8976FE                  	mov word [bp + ?table], si
   461 000002B7 81FE[0C00]              	cmp si, strict word hooktable_end
   462                                  internaldatarelocation
   463 000002BB 7292                    	jb .loop_table
   464                                  
   465                                  
   466 000002BD 8026[1000]FE            	clropt [code + eldiFlags], eldifResident
   467                                  internalcoderelocation -3	; mark block as free
   468 000002C2 BA[2E00]                	mov dx, msg.uninstall_done
   469                                  internaldatarelocation
   470                                  @@:
   471 000002C5 89EC5D                  	lleave
   472 000002C8 16                      	push ss
   473 000002C9 1F                      	pop ds
   474 000002CA E87300                  	extcallcall putsz
   475 000002CD E83800                  	extcallcall cmd3	; return
   476                                  
   477                                  .error:
   478 000002D0 B8010E                  	mov ax, 0E01h
   479 000002D3 E87200                  	extcallcall setrc
   480 000002D6 BA[4600]                	mov dx, msg.uninstall_error
   481                                  internaldatarelocation
   482 000002D9 EBEA                    	jmp @B
   483                                  
   484                                  
   485                                  get_es_ext:
   486 000002DB 8E06[0000]              	mov es, word [relocateddata]
   487                                  linkdatarelocation extdssel
   488 000002DF E86E00                  	extcallcall ispm
   489 000002E2 7404                    	jz @F
   490 000002E4 8E06[0000]              	mov es, word [relocateddata]
   491                                  linkdatarelocation extseg
   492                                  @@:
   493 000002E8 C3                      	retn
   494                                  
   495                                  
   496 000002E9 90<rep 7h>E8[0000]-     	eldcall_dump_callcall ELDCALL_CALLCALL_LIST
   496 000002F3 EB020000C3E8[0000]-
   496 000002FB EB020000C3E8[0000]-
   496 00000303 EB020000C3E8[0000]-
   496 0000030B EB020000C3E8[0000]-
   496 00000313 EB020000C3E8[0000]-
   496 0000031B EB020000C3E8[0000]-
   496 00000323 EB020000C3E8[0000]-
   496 0000032B EB020000C3E8[0000]-
   496 00000333 EB020000C3E8[0000]-
   496 0000033B EB020000C3E8[0000]-
   496 00000343 EB020000C3E8[0000]-
   496 0000034B EB020000C3E8[0000]-
   496 00000353 EB020000C3         
   497                                  
   498                                  endinstalled equ ($ + CODEFIXUP + 15) & ~15
   499                                  
   500                                  
   501                                  start:
   502 00000358 8CC3                    	mov bx, es
   503 0000035A 16                      	 push ss
   504 0000035B 07                      	 pop es
   505 0000035C E891FF                  	call skipcomma
   506 0000035F 4E                      	dec si
   507 00000360 BA[0000]                	mov dx, relocateddata
   508                                  linkdatarelocation msg.install
   509 00000363 E892FF                  	call isstring?
   510 00000366 7433                    	je install
   511 00000368 BA[4D01]                	mov dx, msg.help
   512                                  internaldatarelocation
   513 0000036B E8[0000]EB020000        	extcall putsz
   514 00000372 E80300                  	call uninstall_oneshot
   515 00000375 31C0                    	xor ax, ax
   516 00000377 CB                      	retf
   517                                  
   518                                  
   519                                  uninstall_oneshot:
   520 00000378 36F606[0000]01          	testopt [ss:relocateddata], 1
   521                                  linkdatarelocation options7, -3
   522 0000037E 751A                    	jnz @F
   523                                  
   524 00000380 2EA1[0200]              	mov ax, word [cs:code + eldiEndCode]
   525                                  internalcoderelocation
   526 00000384 2E2B06[0000]            	sub ax, word [cs:code + eldiStartCode]
   527                                  internalcoderelocation
   528 00000389 2906[0000]              	sub word [relocateddata], ax
   529                                  linkdatarelocation extseg_used
   530                                  
   531 0000038D 2EA1[0600]              	mov ax, word [cs:code + eldiEndData]
   532                                  internalcoderelocation
   533 00000391 2E2B06[0400]            	sub ax, word [cs:code + eldiStartData]
   534                                  internalcoderelocation
   535 00000396 2906[0000]              	sub word [relocateddata], ax
   536                                  linkdatarelocation extdata_used
   537                                  @@:
   538 0000039A C3                      	retn
   539                                  
   540                                  
   541                                  DATAOFFSET equ CODEOFFSET + code_size
   542                                  	addsection DATA, follows=CODE vstart=_ELD_DATA_VSTART
   543                                  %define DATAFIXUP - datastart + 0
   544                                  datastart:
   545                                  PUT_ELD_DATETIME
   546                                  
   547                                  	struc HOOKTABLE
   548 00000000 ????                    htEntry:		resw 1
   549 00000002 ????                    htHandler:		resw 1
   550 00000004 ????                    htInstalled:		resw 1
   551                                  	endstruc
   552                                  
   553                                  	align 2, db 0
   554                                  hooktable:
   555                                  		; command last so uninstall abort will leave command installed
   556                                  	istruc HOOKTABLE
   557 00000000 [6800]                  at htEntry,		dw puts_handler
   558                                  internalcoderelocation
   559 00000002 [0000]                  at htHandler,		dw relocateddata
   560                                  linkdatarelocation ext_puts_handler
   561 00000004 0000                    at htInstalled,		dw 0
   562                                  	iend
   563                                  	istruc HOOKTABLE
   564 00000006 [2000]                  at htEntry,		dw command
   565                                  internalcoderelocation
   566 00000008 [0000]                  at htHandler,		dw relocateddata
   567                                  linkdatarelocation ext_command_handler
   568 0000000A 0000                    at htInstalled,		dw 0
   569                                  	iend
   570                                  hooktable_end:
   571                                  
   572                                  	align 2, db 0
   573                                  table:
   574 0000000C [6C00]                  	dw msg.jmp
   575                                  internaldatarelocation
   576 0000000E [7000]                  	dw msg.retn
   577                                  internaldatarelocation
   578 00000010 [7500]                  	dw msg.retf
   579                                  internaldatarelocation
   580 00000012 [7A00]                  	dw msg.iret
   581                                  internaldatarelocation
   582 00000014 0000                    	dw 0
   583                                  
   584                                  width:
   585 00000016 2700                    	dw 39
   586                                  
   587                                  ah_4Ch_table:
   588 00000018 [8900]                  	dw msg.mov
   589                                  internaldatarelocation
   590 0000001A [8D00]                  	dw msg.ah
   591                                  internaldatarelocation
   592 0000001C [8900]                  	dw msg.mov
   593                                  internaldatarelocation
   594 0000001E [9000]                  	dw msg.ax
   595                                  internaldatarelocation
   596 00000020 0000                    	dw 0
   597                                  
   598                                  mov_ah_4Ch:
   599 00000022 00                      	db 0
   600                                  isregdump:
   601 00000023 00                      	db 0
   602                                  wasregdump:
   603 00000024 00                      	db 0
   604                                  
   605                                  msg:
   606 00000025 555345504152415400      .useparat:		asciz "USEPARAT"
   607 0000002E 555345504152415420-     .uninstall_done:	db "USEPARAT uninstalled."
   607 00000037 756E696E7374616C6C-
   607 00000040 65642E             
   608                                  %if _ELD_RECLAIM_HINT
   609                                  			db " (Don't forget to use reclaim.eld)"
   610                                  %endif
   611 00000043 0D0A00                  			asciz 13,10
   612 00000046 555345504152415420-     .uninstall_error:	asciz "USEPARAT unable to uninstall!",13,10
   612 0000004F 756E61626C6520746F-
   612 00000058 20756E696E7374616C-
   612 00000061 6C210D0A00         
   613 00000066 574944544800            .width:	asciz "WIDTH"
   614 0000006C 4A4D5000                .jmp:	asciz "JMP"
   615 00000070 5245544E00              .retn:	asciz "RETN"
   616 00000075 5245544600              .retf:	asciz "RETF"
   617 0000007A 4952455400              .iret:	asciz "IRET"
   618 0000007F 494E5400                .int:	asciz "INT"
   619 00000083 323000                  .20:	asciz "20"
   620 00000086 323100                  .21:	asciz "21"
   621 00000089 4D4F5600                .mov:	asciz "MOV"
   622 0000008D 414800                  .ah:	asciz "AH"
   623 00000090 415800                  .ax:	asciz "AX"
   624 00000093 5F<rep 50h>             .separator:		times 80 db "_"
   625 000000E3 0D0A                    .separator_linebreak:	db 13,10
   626                                  endarea .separator_linebreak
   627 000000E5 3D<rep 50h>             .separator_terminate:	times 80 db "="
   628 00000135 0D0A                    			db 13,10
   629                                  
   630                                  uinit_data: equ $
   631                                  
   632 00000137 555345504152415420-     .installed:	asciz "USEPARAT installed.",13,10
   632 00000140 696E7374616C6C6564-
   632 00000149 2E0D0A00           
   633 0000014D 496E7374616C6C2074-     .help:		db "Install this ELD using an INSTALL keyword.",13,10
   633 00000156 68697320454C442075-
   633 0000015F 73696E6720616E2049-
   633 00000168 4E5354414C4C206B65-
   633 00000171 79776F72642E0D0A   
   634 00000179 0D0A                    		db 13,10
   635 0000017B 507574732073657061-     		db "Puts separators in disassembly on control flow end.",13,10
   635 00000184 7261746F727320696E-
   635 0000018D 20646973617373656D-
   635 00000196 626C79206F6E20636F-
   635 0000019F 6E74726F6C20666C6F-
   635 000001A8 7720656E642E0D0A   
   636 000001B0 41206C696E65206F66-     		db "A line of underscores is inserted after disassembly of far or near jump,",13,10
   636 000001B9 20756E64657273636F-
   636 000001C2 72657320697320696E-
   636 000001CB 736572746564206166-
   636 000001D4 746572206469736173-
   636 000001DD 73656D626C79206F66-
   636 000001E6 20666172206F72206E-
   636 000001EF 656172206A756D702C-
   636 000001F8 0D0A               
   637 000001FA 6F7220696E74657272-     		db "or interrupt, far, or near return.",13,10
   637 00000203 7570742C206661722C-
   637 0000020C 206F72206E65617220-
   637 00000215 72657475726E2E0D0A 
   638 0000021E 41206C696E65206F66-     		db "A line of equals signs is inserted after detecting a DOS termination call.",13,10
   638 00000227 20657175616C732073-
   638 00000230 69676E732069732069-
   638 00000239 6E7365727465642061-
   638 00000242 667465722064657465-
   638 0000024B 6374696E6720612044-
   638 00000254 4F53207465726D696E-
   638 0000025D 6174696F6E2063616C-
   638 00000266 6C2E0D0A           
   639 0000026A 285468652064657465-     		db "(The detection is not perfect.)",13,10
   639 00000273 6374696F6E20697320-
   639 0000027C 6E6F74207065726665-
   639 00000285 63742E290D0A       
   640 0000028B 0D0A                    		db 13,10
   641 0000028D 52756E207769746820-     		db "Run with USEPARAT WIDTH expression to set width (0 to #80, default #39).",13,10
   641 00000296 555345504152415420-
   641 0000029F 574944544820657870-
   641 000002A8 72657373696F6E2074-
   641 000002B1 6F2073657420776964-
   641 000002BA 746820283020746F20-
   641 000002C3 2338302C2064656661-
   641 000002CC 756C7420233339292E-
   641 000002D5 0D0A               
   642 000002D7 52756E207769746820-     		db "Run with USEPARAT UNINSTALL to uninstall.",13,10
   642 000002E0 555345504152415420-
   642 000002E9 554E494E5354414C4C-
   642 000002F2 20746F20756E696E73-
   642 000002FB 74616C6C2E0D0A     
   643 00000302 00                      		asciz
   644                                  
   645                                  
   646 00000303 00<rep Dh>              	align 16, db 0
   647                                  init_data_end:
   648                                  data_size equ $ - datastart
   649                                  transient_data_size equ data_size
   650                                  
   651                                  	absolute uinit_data
   652                                  
   653 00000137 <res 9h>                	alignb 16
   654                                  uinit_data_end:
   655                                  resident_data_end:
   656                                  resident_data_size equ resident_data_end - datastart
   657                                  
   658                                  %if uinit_data_end >= init_data_end
   659                                   total_data_size equ $ - datastart
   660                                  %else
   661                                   total_data_size equ init_data_end - datastart
   662                                  %endif
   663                                  %assign _DATA_SIZE total_data_size
   664                                  
   665                                  
   666                                  	usesection CODE
   667                                  
   668                                  install:
   669 0000039B AC                      	lodsb
   670 0000039C E8[0000]EB020000        	extcall chkeol
   671                                  
   672                                  	houdini
   673 000003A3 8EC3                    	mov es, bx		; => ext seg (writable)
   674                                  
   675 000003A5 B8A000                  	mov ax, endresident - endinstalled
   676 000003A8 262906[0200]            	sub word [es:code + eldiEndCode], ax
   677                                  internalcoderelocation		; adjust size
   678 000003AD 2906[0000]              	sub word [relocateddata], ax
   679                                  linkdatarelocation extseg_used	; adjust size
   680                                  
   681                                  %if (transient_data_size - resident_data_size) > 0
   682 000003B1 B8D001                  	mov ax, transient_data_size - resident_data_size
   683 000003B4 262906[0600]            	sub word [es:code + eldiEndData], ax
   684                                  internalcoderelocation		; adjust size
   685 000003B9 2906[0000]              	sub word [relocateddata], ax
   686                                  linkdatarelocation extdata_used	; adjust size
   687                                  %endif
   688                                  
   689 000003BD BE[0600]                	mov si, hooktable_end - HOOKTABLE_size
   690                                  internaldatarelocation
   691                                  
   692                                  .loop_table:
   693 000003C0 8B5C02                  	mov bx, word [si + htHandler]; -> handler
   694 000003C3 8B1F                    	mov bx, word [bx]	; -> prior
   695 000003C5 8B3C                    	mov di, word [si + htEntry]	; -> our handler
   696 000003C7 85DB                    	test bx, bx		; installing as first ?
   697 000003C9 740A                    	jz .only_first		; yes, simple --> (leave as extcall cmd3_not_ext)
   698 000003CB AF                      	scasw			; skip entrypoint jmp strict short
   699 000003CC B0E9                    	mov al, 0E9h		; = jmp near opcode
   700 000003CE AA                      	stosb			; store
   701 000003CF 93                      	xchg ax, bx		; ax -> next handler
   702 000003D0 29F8                    	sub ax, di
   703 000003D2 48                      	dec ax
   704 000003D3 48                      	dec ax			; ax = ax - (di + 2)
   705 000003D4 AB                      	stosw			; store our downlink as rel16 displacement
   706                                  
   707                                  .only_first:
   708 000003D5 8B5C02                  	mov bx, word [si + htHandler]; -> handler
   709 000003D8 8B04                    	mov ax, word [si + htEntry]
   710 000003DA 8907                    	mov word [bx], ax	; -> our entrypoint
   711 000003DC F65404                  	not byte [si + htInstalled]
   712                                  
   713                                  .next_table:
   714 000003DF 83EE06                  	sub si, HOOKTABLE_size
   715 000003E2 81FE[0000]              	cmp si, strict word hooktable
   716                                  internaldatarelocation
   717 000003E6 73D8                    	jae .loop_table
   718                                  
   719 000003E8 26800E[1000]01          	setopt [es:code + eldiFlags], eldifResident
   720                                  internalcoderelocation -3	; mark block as resident
   721                                  
   722 000003EE F606[0000]04            	testopt [relocateddata], 4
   723                                  linkdatarelocation options7, -3
   724 000003F3 7506                    	jnz @F
   725 000003F5 BA[3701]                	mov dx, msg.installed
   726                                  internaldatarelocation
   727 000003F8 E845FF                  	call putsz
   728                                  @@:
   729 000003FB 31C0                    	xor ax, ax
   730 000003FD CB                      	retf
   731                                  
   732                                  
   733                                  %include "eldlink.asm"
     1                              <1> %if 0
     2                              <1> 
     3                              <1> Extensions for lDebug linker
     4                              <1> 
     5                              <1> Copyright (C) 2008-2025 E. C. Masloch
     6                              <1> 
     7                              <1> Usage of the works is permitted provided that this
     8                              <1> instrument is retained with the works, so that any entity
     9                              <1> that uses the works is notified of this instrument.
    10                              <1> 
    11                              <1> DISCLAIMER: THE WORKS ARE WITHOUT WARRANTY.
    12                              <1> 
    13                              <1> %endif
    14                              <1> 
    15                              <1> %include "lmacros3.mac"
     1                              <2> [list -]
    16                              <1> %include "eld.mac"
     1                              <2> %if 0
     2                              <2> 
     3                              <2> Extensions for lDebug macros
     4                              <2> 
     5                              <2> Copyright (C) 2008-2025 E. C. Masloch
     6                              <2> 
     7                              <2> Usage of the works is permitted provided that this
     8                              <2> instrument is retained with the works, so that any entity
     9                              <2> that uses the works is notified of this instrument.
    10                              <2> 
    11                              <2> DISCLAIMER: THE WORKS ARE WITHOUT WARRANTY.
    12                              <2> 
    13                              <2> %endif
    14                              <2> 
    15                              <2> %ifndef ELD_MAC
    16                              <2> %define ELD_MAC 1
    17                              <2> 
    18                              <2> %include "lmacros3.mac"
    19                              <2> 
    20                              <2> 		; ELD executable header
    21                              <2> 	struc ELD_HEADER
    22                              <2> eldhSignature:		resb 4	; "ELD1"
    23                              <2> 			resb 3	; reserved
    24                              <2> 			resb 1	; 26 (Ctrl-Z)
    25                              <2> eldhCodeOffset:		resd 1	; position displacement from eldhSignature
    26                              <2> eldhCodeImageLength:	resw 1	; amount bytes, at least 32
    27                              <2> eldhCodeAllocLength:	resw 1	; amount bytes, added to prior. sum < 64 KiB
    28                              <2> eldhDataOffset:		resd 1
    29                              <2> eldhDataImageLength:	resw 1	; (zero allowed)
    30                              <2> eldhDataAllocLength:	resw 1	; (zero allowed)
    31                              <2> eldhCodeEntrypoint:	resw 1	; within code section, used as displacement
    32                              <2> eldhReserved:		resb 4	; reserved
    33                              <2> eldhExtensionSize:	resw 1	; from eldhSignature, -> past eldhx fields in use
    34                              <2> 	endstruc
    35                              <2> 	endarea ELD_HEADER, 1
    36                              <2> 
    37                              <2> 	struc ELD_HEADERX
    38                              <2> eldhxHeader:		resb ELD_HEADER_size
    39                              <2> eldhxDescriptionOffset:	resd 1	; zero if none, from eldhxHeader. <= 128 Bytes
    40                              <2> eldhxHelpOffset:	resd 1	; zero if none, from eldhxHeader
    41                              <2> eldhxLibTable:		resd 1	; zero if none, from eldhxHeader
    42                              <2> eldhxDateTimeOffset:	resd 1	; zero if none, from eldhxHeader
    43                              <2> 	alignb 16
    44                              <2> 	endstruc
    45                              <2> 
    46                              <2> 	struc ELD_TRAILER_HEADER
    47                              <2> eldthSignature:		resb 8	; "ELD1TAIL"
    48                              <2> eldthHeaderOffset:	resd 1	; negative displacement from eldthSignature,
    49                              <2> 				;  add this dword to the seek offset
    50                              <2> eldthReserved:		resw 1	; reserved, must be initialised to zero
    51                              <2> eldthChecksum:		resw 1	; sum of all words in trailer header = 0
    52                              <2> 	endstruc
    53                              <2> 	endarea ELD_TRAILER_HEADER, 1
    54                              <2> 
    55                              <2> 	struc ELD_LIBTABLE
    56                              <2> eldltFormat:		resw 1
    57                              <2> 	; 0 = uncompressed
    58                              <2> 	; 2 = heatshrink compressed
    59                              <2> 	; 3 = lzexedat -4 compressed
    60                              <2> 	; 4 = lzexedat -4 -l compressed
    61                              <2> eldltAmount:		resw 1
    62                              <2> eldltOffset:		resd 1	; from eldhxHeader
    63                              <2> eldltCompressedLength:		; (dword, only present if format 2, 3, or 4)
    64                              <2> 	endstruc
    65                              <2> 	endarea ELD_LIBTABLE, 1
    66                              <2> 
    67                              <2> 		; ELD instance header
    68                              <2> 	struc ELD_INSTANCE
    69                              <2> eldiStartCode:		resw 1	; -> this structure itself (para aligned)
    70                              <2> eldiEndCode:		resw 1	; -> behind memory used by instance (para aligned)
    71                              <2> eldiStartData:		resw 1	; -> data in data entry section (para aligned), or 0
    72                              <2> eldiEndData:		resw 1	; -> behind data (para aligned), or 0
    73                              <2> eldiIdentifier:		resb 8	; blank-filled text
    74                              <2> eldiFlags:		resw 1	; flags
    75                              <2> eldiListing_size equ 14
    76                              <2> eldiListing:		resb eldiListing_size
    77                              <2> 				; ASCIZ listing file name
    78                              <2> 	endstruc
    79                              <2> 		; flags for eldiFlags:
    80                              <2> eldifResident:		equ 1
    81                              <2> 
    82                              <2> 		; ELD link info header
    83                              <2> 	struc ELD_LINKINFO
    84                              <2> eldlSignature:		resw 1	; 0E1D1h
    85                              <2> eldlReserved:		resw 2
    86                              <2> eldlUseLinkHash:	resw 1
    87                              <2> eldlDataAmount:		resw 1
    88                              <2> eldlDataPrefixes:	resw 1
    89                              <2> eldlDataEntries:	resw 1
    90                              <2> eldlDataAddresses:	resw 1
    91                              <2> eldlCodeAmount:		resw 1
    92                              <2> eldlCodePrefixes:	resw 1
    93                              <2> eldlCodeEntries:	resw 1
    94                              <2> eldlCodeAddresses:	resw 1
    95                              <2> 	endstruc
    96                              <2> 
    97                              <2> 	numdef ELD_CODE_VSTART, 9001h
    98                              <2> 	numdef ELD_DATA_VSTART, 8000h
    99                              <2> 	numdef ELD_RELOC_VSTART, 8000h
   100                              <2> 
   101                              <2> 	numdef ELD_RECLAIM_HINT, 0
   102                              <2> 	strdef ELD_LISTING, ""
   103                              <2> 	numdef ELD_DATETIME, 0
   104                              <2> 
   105                              <2> %if _ELD_DATETIME
   106                              <2>  %define PUT_ELDHX_DATETIME_OFFSET at eldhxDateTimeOffset, dd DATAOFFSET + datetime - datastart
   107                              <2>  %macro PUT_ELD_DATETIME 0.nolist
   108                              <2> datetime:	asciz __UTC_DATE__,'T',__UTC_TIME__,'Z'
   109                              <2> 		asciz		; for future extension
   110                              <2>  %endmacro
   111                              <2> %else
   112                              <2>  %define PUT_ELDHX_DATETIME_OFFSET
   113                              <2>  %define PUT_ELD_DATETIME
   114                              <2> %endif
   115                              <2> 
   116                              <2> %endif
    17                              <1> 
    18                              <1> 	cpu 8086
    19                              <1> 
    20                              <1> %if ELDSTRICT
    21                              <1>  %if ELDSTRICTCOUNTER
    22                              <1>   %error Missing relocation
    23                              <1>  %endif
    24                              <1> %endif
    25                              <1> 	eldstrict off		; linker does some relocations
    26                              <1> 
    27                              <1> %ifn ELDCALLCALL_DUMPED
    28                              <1> 	eldcall_dump_callcall ELDCALL_CALLCALL_LIST
    29                              <1> %endif
    30                              <1> 
    31                              <1> 	numdef ELD_IDENTICALISE, 0
    32                              <1> 	numdef ELD_DEBUG, 0
    33                              <1> 	numdef ELD_LINKER_PASSES, 1
    34                              <1> 	strdef LISTING, _ELD_LISTING
    35                              <1> 	numdef ELDCALL_OPTIONAL, ELDCALL_OPTIONAL_STATUS
    36                              <1> 	numdef ELDDATA_OPTIONAL, ELDDATA_OPTIONAL_STATUS
    37                              <1> %if _ELD_IDENTICALISE
    38                              <1>  ;%assign _ELDCALL_OPTIONAL 1
    39                              <1> %endif
    40                              <1> %ifn _ELDCALL_OPTIONAL
    41                              <1> %assign ELDCALL_OPTIONAL_STATUS 2		; not allowed
    42                              <1> %endif
    43                              <1> ;%ifn _ELDDATA_OPTIONAL
    44                              <1> ;%assign ELDDATA_OPTIONAL_STATUS 2		; not allowed
    45                              <1> ;%endif
    46                              <1> 	gendef MAP, ""
    47                              <1> 
    48                              <1> %ifnidni _MAP, ""
    49                              <1>  [map all _MAP]
    50                              <1> %endif
    51                              <1> 
    52                              <1> 
    53                              <1> endresident: equ ($ + _CURRENT_SECTION %+ FIXUP + 15) & ~15
    54                              <1> 
    55                              <1> %if _ELD_LINKER_PASSES
    56                              <1> %assign ELDLINKER 1
    57                              <1> 
    58                              <1> 	struc LINKTABLE
    59 00000000 ????????            <1> ltCodeToCode:	resw 2
    60 00000004 ????????            <1> ltCodeToData:	resw 2
    61 00000008 ????????            <1> ltDataToCode:	resw 2
    62 0000000C ????????            <1> ltDataToData:	resw 2
    63 00000010 ????????            <1> ltLinkData:	resw 2
    64 00000014 ????????            <1> ltLinkCode:	resw 2
    65                              <1> 	endstruc
    66                              <1> %endif
    67                              <1> 
    68                              <1> 
    69                              <1> 		; INP:	es:dx -> loaded initial ELD image
    70                              <1> 		;	 ELD instance structure filled
    71                              <1> 		;	es => ELD code area
    72                              <1> 		;	ds:di -> link info
    73                              <1> 		;	ss:bx -> loaded initial data
    74                              <1> 		;	ss:si -> command line tail
    75                              <1> 		;	cs:ip -> entrypoint
    76                              <1> 		;	ss:sp -> far return address for current mode
    77                              <1> 		; STT:	UP, EI
    78                              <1> linker:
    79                              <1> 		; The first 15 Bytes of the linker should be
    80                              <1> 		;  the same regardless of the linker options
    81                              <1> 		;  used (debug, passes, vstart). This allows
    82                              <1> 		;  the eldcomp ELD to match even if up to 15
    83                              <1> 		;  Bytes of the linker are trailing in the
    84                              <1> 		;  resident part of the ELD.
    85                              <1> 	lframe
    86                              <1>  %if ELDOTHER
    87                              <1> 	lvar dword, linkinfo_other
    88                              <1> 	lvar word, use_hash_other
    89                              <1>  %endif
    90 000003FE 5589E5              <1> 	lenter
    91                              <1> 	lvar dword, instance
    92 00000401 06                  <1> 	 push es
    93 00000402 52                  <1> 	 push dx		; -> start of where we're loaded in ELD cs
    94                              <1> 	lvar word, targetsection_low_optional_high
    95 00000403 50                  <1> 	 push ax		; placeholder
    96                              <1> 	lequ ?targetsection_low_optional_high, targetsection
    97                              <1> 	lequ ?targetsection_low_optional_high + 1, optional
    98                              <1> 	lvar dword, linkinfo
    99 00000404 1E                  <1> 	 push ds
   100 00000405 57                  <1> 	 push di		; -> link info (in debugger ss or message seg)
   101                              <1> 	lvar dword, nextreloc
   102 00000406 06                  <1> 	 push es		; => ELD cs
   103 00000407 52                  <1> 	 push dx		; placeholder
   104                              <1> 	lvar dword, entry
   105 00000408 06                  <1> 	 push es		; => ELD cs
   106 00000409 50                  <1> 	 push ax		; placeholder
   107 0000040A 31C0                <1> 	xor ax, ax
   108 0000040C 813DD1E1            <1> 	cmp word [di + eldlSignature], 0E1D1h
   109                              <1> %if ($ - linker) < 16
   110                              <1>  %error Expected invariant first paragraph of linker
   111                              <1> %endif
   112 00000410 7403E95E02          <1> 	jne .error_j		; signature mismatch -->
   113 00000415 837D0601            <1> 	cmp word [di + eldlUseLinkHash], 1
   114 00000419 7603E95502          <1> 	ja .error_j		; unknown use link hash number -->
   115 0000041E 7201                <1> 	jb @F
   116 00000420 48                  <1> 	dec ax			; = -1 if hash used
   117                              <1> @@:
   118                              <1> 	lvar word, use_hash
   119 00000421 50                  <1> 	 push ax		; = -1 if hash used, else 0
   120                              <1> %if _ELD_IDENTICALISE && _ELD_LINKER_PASSES
   121                              <1> 	mov ax, linktable - code
   122                              <1> 	lvar word, lt
   123                              <1> 	 push ax		; -> link tables (a single reference)
   124                              <1> %endif
   125                              <1> %if _ELD_LINKER_PASSES || ELDOTHER
   126 00000422 31C0                <1> 	xor ax, ax
   127                              <1>  %if _ELD_LINKER_PASSES
   128                              <1> 	lvar word, pass
   129 00000424 50                  <1> 	 push ax		; = 0 for linker itself, = 2 for application
   130                              <1> 	lvar word, amounterrors
   131 00000425 50                  <1> 	 push ax		; how many distinct errors encountered in pass 2
   132                              <1> 	lvar word, name
   133 00000426 50                  <1> 	 push ax		; -> name currently being sought (in our table)
   134                              <1>  %endif
   135                              <1>  %if ELDOTHER
   136                              <1> 	lvar word, other
   137                              <1> 	 push ax		; byte: 0 = own data links, -1 = other data links
   138                              <1>  %endif
   139                              <1> %endif
   140 00000427 56                  <1> 	push si			; -> command line tail
   141 00000428 53                  <1> 	push bx			; -> data block in ELD data area (segment ss)
   142                              <1> 
   143                              <1> 			; simple: add instance base (dx) to code
   144 00000429 06                  <1> 	push es
   145 0000042A 1F                  <1> 	pop ds			; ds = es => ELD cs
   146                              <1> %if _ELD_LINKER_PASSES
   147                              <1> .pass:
   148 0000042B 8B5EEA              <1> 	mov bx, word [bp + ?pass]	; 0 or 2
   149 0000042E 01D3                <1> 	add bx, dx		; -> start of the ELD instance in cs, +0 or +2
   150                              <1>  %if _ELD_IDENTICALISE
   151                              <1> 	add bx, word [bp + ?lt]	; add in single reference to linktable
   152                              <1> 	mov si, word [ltCodeToCode + bx]
   153                              <1>  %else
   154 00000430 8BB7B407            <1> 	mov si, word [linktable - code + ltCodeToCode + bx]
   155                              <1>  %endif
   156                              <1> %else
   157                              <1> 	mov si, internalcodetocoderelocations - code
   158                              <1> %endif		 		; si -> table for code to code (linker or app)
   159 00000434 01D6                <1> 	add si, dx		; relocate the table pointer itself
   160                              <1> @@:
   161 00000436 AD                  <1> 	lodsw
   162 00000437 85C0                <1> 	test ax, ax		; was last ?
   163 00000439 740B                <1> 	jz @F			; yes -->
   164 0000043B 93                  <1> 	xchg bx, ax		; bx = entry
   165 0000043C 01D3                <1> 	add bx, dx		; relocate the entry itself
   166                              <1> %if _ELD_CODE_VSTART
   167 0000043E 812F[0000]          <1> 	sub word [bx], code	; undo adjustment
   168                              <1> %endif
   169 00000442 0117                <1> 	add word [bx], dx	; relocate word referenced by entry
   170 00000444 EBF0                <1> 	jmp @B
   171                              <1> 
   172                              <1> @@:
   173                              <1> 			; next, add heap data base (on stack) to code
   174                              <1> %if _ELD_LINKER_PASSES
   175 00000446 8B5EEA              <1> 	mov bx, word [bp + ?pass]	; 0 or 2
   176 00000449 01D3                <1> 	add bx, dx		; -> start of the ELD instance in cs, +0 or +2
   177                              <1>  %if _ELD_IDENTICALISE
   178                              <1> 	add bx, word [bp + ?lt]	; add in single reference to linktable
   179                              <1> 	mov si, word [ltCodeToData + bx]
   180                              <1>  %else
   181 0000044B 8BB7B807            <1> 	mov si, word [linktable - code + ltCodeToData + bx]
   182                              <1>  %endif
   183                              <1> %else
   184                              <1> 	mov si, internalcodetodatarelocations - code
   185                              <1> %endif				; si -> table for code to data (linker or app)
   186 0000044F 01D6                <1> 	add si, dx		; relocate the table pointer itself
   187                              <1> @@:
   188 00000451 AD                  <1> 	lodsw
   189 00000452 85C0                <1> 	test ax, ax		; was last ?
   190 00000454 740C                <1> 	jz @F			; yes -->
   191 00000456 93                  <1> 	xchg bx, ax		; bx = entry
   192 00000457 01D3                <1> 	add bx, dx		; relocate the entry itself
   193                              <1> 		; ! access the offset of the data area block, topmost on stack
   194 00000459 58                  <1> 	pop ax			; ax -> heap data
   195 0000045A 50                  <1> 	push ax
   196                              <1> %if _ELD_DATA_VSTART
   197 0000045B 2D[0000]            <1> 	sub ax, datastart	; undo adjustment
   198                              <1> %endif
   199 0000045E 0107                <1> 	add word [bx], ax	; relocate word referenced by entry
   200 00000460 EBEF                <1> 	jmp @B
   201                              <1> 
   202                              <1> @@:
   203                              <1> 
   204                              <1> 			; add instance base (dx) to data
   205                              <1> %if _ELD_LINKER_PASSES
   206 00000462 8B5EEA              <1> 	mov bx, word [bp + ?pass]
   207 00000465 01D3                <1> 	add bx, dx
   208                              <1>  %if _ELD_IDENTICALISE
   209                              <1> 	add bx, word [bp + ?lt]
   210                              <1> 	mov si, word [ltDataToCode + bx]
   211                              <1>  %else
   212 00000467 8BB7BC07            <1> 	mov si, word [linktable - code + ltDataToCode + bx]
   213                              <1>  %endif
   214                              <1> %else
   215                              <1> 	mov si, internaldatatocoderelocations - code
   216                              <1> %endif
   217 0000046B 01D6                <1> 	add si, dx
   218                              <1> @@:
   219 0000046D AD                  <1> 	lodsw
   220 0000046E 83F8FF              <1> 	cmp ax, -1		; was last ?
   221 00000471 740F                <1> 	je @F			; yes -->
   222 00000473 93                  <1> 	xchg bx, ax		; bx = entry
   223                              <1> 		; ! access the offset of the data area block, topmost on stack
   224 00000474 58                  <1> 	pop ax
   225 00000475 50                  <1> 	push ax
   226 00000476 01C3                <1> 	add bx, ax		; relocate the entry itself
   227                              <1> %if _ELD_CODE_VSTART
   228 00000478 36812F[0000]        <1> 	sub word [ss:bx], code	; undo adjustment
   229                              <1> %endif
   230 0000047D 360117              <1> 	add word [ss:bx], dx	; relocate word referenced by entry
   231 00000480 EBEB                <1> 	jmp @B
   232                              <1> 
   233                              <1> @@:
   234                              <1> 			; next, add heap data base (on stack) to data
   235                              <1> %if _ELD_LINKER_PASSES
   236 00000482 8B5EEA              <1> 	mov bx, word [bp + ?pass]
   237 00000485 01D3                <1> 	add bx, dx
   238                              <1>  %if _ELD_IDENTICALISE
   239                              <1> 	add bx, word [bp + ?lt]
   240                              <1> 	mov si, word [ltDataToData + bx]
   241                              <1>  %else
   242 00000487 8BB7C007            <1> 	mov si, word [linktable - code + ltDataToData + bx]
   243                              <1>  %endif
   244                              <1> %else
   245                              <1> 	mov si, internaldatatodatarelocations - code
   246                              <1> %endif
   247 0000048B 01D6                <1> 	add si, dx
   248                              <1> @@:
   249 0000048D AD                  <1> 	lodsw
   250 0000048E 83F8FF              <1> 	cmp ax, -1		; was last ?
   251 00000491 740D                <1> 	je @F			; yes -->
   252 00000493 93                  <1> 	xchg bx, ax		; bx = entry
   253                              <1> 		; ! access the offset of the data area block, topmost on stack
   254 00000494 58                  <1> 	pop ax			; ax -> heap data
   255 00000495 50                  <1> 	push ax
   256 00000496 01C3                <1> 	add bx, ax		; relocate the entry itself
   257                              <1> %if _ELD_DATA_VSTART
   258 00000498 2D[0000]            <1> 	sub ax, datastart	; undo adjustment
   259                              <1> %endif
   260 0000049B 360107              <1> 	add word [ss:bx], ax	; relocate word referenced by entry
   261 0000049E EBED                <1> 	jmp @B
   262                              <1> 
   263                              <1> @@:
   264 000004A0 8B56FC              <1> 	mov dx, word [bp + ?instance]
   265                              <1> 				; reset (why??) -> ELD instance in ELD cs
   266                              <1> %if _ELD_LINKER_PASSES
   267 000004A3 8B5EEA              <1> 	mov bx, word [bp + ?pass]
   268 000004A6 01D3                <1> 	add bx, dx
   269                              <1>  %if _ELD_IDENTICALISE
   270                              <1> 	add bx, word [bp + ?lt]
   271                              <1> 	add dx, word [ltLinkData + bx]
   272                              <1>  %else
   273 000004A8 0397C407            <1> 	add dx, word [linktable - code + ltLinkData + bx]
   274                              <1>  %endif
   275                              <1> %else
   276                              <1> 	add dx, linkerdatarelocations - code
   277                              <1> %endif
   278                              <1> .otherloop:
   279 000004AC 8956F2              <1> 	mov word [bp + ?nextreloc], dx
   280                              <1> 				; -> data link relocation table
   281                              <1> 
   282                              <1> .datarelocloop:		; must be done before further relocs
   283 000004AF C576F2              <1> 	lds si, [bp + ?nextreloc]
   284 000004B2 AD                  <1> 	lodsw			; ax = section indicator
   285 000004B3 85C0                <1> 	test ax, ax		; end of table ?
   286 000004B5 7503E92601          <1> 	jz .donedatareloc
   287 000004BA 48                  <1> 	dec ax			; al = 1 if data, 0 if code (NB ah may != 0)
   288                              <1> 		; ! access the offset of the data area block, topmost on stack
   289 000004BB 5B                  <1> 	pop bx
   290 000004BC 53                  <1> 	push bx			; bx -> ELD data block
   291 000004BD 8946FA              <1> 	mov word [bp + ?targetsection_low_optional_high], ax
   292 000004C0 84C0                <1> 	test al, al		; data ?
   293 000004C2 AD                  <1> 	lodsw
   294 000004C3 7504                <1> 	jnz @F			; yes -->
   295 000004C5 0346FC              <1> 	add ax, word [bp + ?instance]
   296                              <1> 				; relocate entry into code
   297 000004C8 A9                  <1> 	db __TEST_IMM16		; (skip add)
   298                              <1> @@:
   299 000004C9 01D8                <1> 	add ax, bx		; relocate entry into data
   300 000004CB 8946EE              <1> 	mov word [bp + ?entry], ax
   301                              <1> 				; save away -> where to patch
   302 000004CE AD                  <1> 	lodsw			; get unrelocated -> name
   303 000004CF 8976F2              <1> 	mov word [bp + ?nextreloc], si
   304                              <1> 				; update -> behind relocation table entry
   305 000004D2 E8DF00              <1> 	call .build_match	; get ax = scan value, si -> counted string,
   306                              <1> 				;  dl = original value at byte [si]
   307                              <1> 				; NC if symbol already not found before
   308                              <1> 				; CY if to search for the symbol
   309                              <1> %if _ELD_LINKER_PASSES
   310 000004D5 73D8                <1> 	jnc .datarelocloop	; if duplicate of a not found symbol -->
   311                              <1> %endif
   312 000004D7 C45EF6              <1> 	les bx, [bp + ?linkinfo]
   313                              <1> %if ELDOTHER
   314                              <1> 	rol byte [bp + ?other], 1
   315                              <1> 	jnc @F
   316                              <1> 	les bx, [bp + ?linkinfo_other]
   317                              <1> @@:
   318                              <1> %endif				; es:bx -> link info table of the ELD host
   319 000004DA 268B4F08            <1> 	mov cx, word [es:bx + eldlDataAmount]	; amount data link info
   320 000004DE 268B7F0A            <1> 	mov di, word [es:bx + eldlDataPrefixes]	; -> prefixes or hashes
   321                              <1> .datarelocfind:
   322 000004E2 83F901              <1> 	cmp cx, 1			; NZ if cx == 0
   323 000004E5 F2AF                <1> 	repne scasw			; scan initial
   324 000004E7 7541                <1> 	jne .datarelocnotfound
   325 000004E9 57                  <1> 	push di
   326 000004EA 51                  <1> 	push cx
   327 000004EB 56                  <1> 	push si
   328 000004EC 262B7F0A            <1> 	sub di, word [es:bx + eldlDataPrefixes]	; = double index, 1-based
   329 000004F0 4F                  <1> 	dec di
   330 000004F1 4F                  <1> 	dec di				; 0-based
   331 000004F2 26037F0C            <1> 	add di, word [es:bx + eldlDataEntries]	; -> entry
   332 000004F6 268B3D              <1> 	mov di, [es:di]			; -> counted suffix/string
   333 000004F9 B500                <1> 	mov ch, 0
   334 000004FB 8A0C                <1> 	mov cl, byte [si]		; cx = length
   335 000004FD 41                  <1> 	inc cx
   336                              <1> 	; cmp al, al			; ZR if length is zero
   337 000004FE F3A6                <1> 	repe cmpsb			; match ?
   338 00000500 5E                  <1> 	pop si
   339 00000501 59                  <1> 	pop cx
   340 00000502 5F                  <1> 	pop di
   341 00000503 75DD                <1> 	jne .datarelocfind		; if not found this time,
   342                              <1> 					;  scan for next initial -->
   343 00000505 8814                <1> 	mov byte [si], dl		; restore the original byte at counter
   344 00000507 262B7F0A            <1> 	sub di, word [es:bx + eldlDataPrefixes]	; = double index, 1-based
   345 0000050B 4F                  <1> 	dec di
   346 0000050C 4F                  <1> 	dec di				; 0-based
   347 0000050D 26037F0E            <1> 	add di, word [es:bx + eldlDataAddresses]	; -> address (offset)
   348 00000511 268B05              <1> 	mov ax, word [es:di]		; get link data from the table
   349 00000514 E80700              <1> 	call .address_data_reloc
   350                              <1> %if _ELD_RELOC_VSTART
   351 00000517 2D[0000]            <1> 	sub ax, relocateddata		; *not* a relocation
   352                              <1> %endif
   353 0000051A 0104                <1> 	add word [si], ax		; relocate
   354 0000051C EB91                <1> 	jmp .datarelocloop
   355                              <1> 
   356                              <1> .address_data_reloc:
   357 0000051E C576EE              <1> 	lds si, [bp + ?entry]		; -> entry if in ELD code instance
   358 00000521 807EFA00            <1> 	cmp byte [bp + ?targetsection], 0
   359                              <1> 					; relocation in code ?
   360 00000525 7402                <1> 	je @F				; yes -->
   361 00000527 16                  <1> 	push ss
   362 00000528 1F                  <1> 	pop ds				; => our ELD data block
   363                              <1> @@:
   364 00000529 C3                  <1> 	retn
   365                              <1> 
   366                              <1> .datarelocnotfound:
   367 0000052A 8814                <1> 	mov byte [si], dl		; restore the original byte at counter
   368 0000052C 807EFB00            <1> 	cmp byte [bp + ?optional], 0	; is it an optional relocation ?
   369                              <1> %if _ELD_DEBUG
   370                              <1> 	jne @F
   371                              <1>  %ifn _ELD_LINKER_PASSES
   372                              <1> 	mov si, 0			; (invalid link)
   373                              <1> linkdatarelocation internalflags6
   374                              <1> 	test si, si
   375                              <1> 	jz .datanotfound
   376                              <1> 	mov si, 0			; (invalid link)
   377                              <1> linkdatarelocation options7
   378                              <1> 	test si, si
   379                              <1> 	jz .datanotfound
   380                              <1>  %else
   381                              <1> 	cmp byte [bp + ?pass], 0
   382                              <1> 	je .datanotfound
   383                              <1>  %endif
   384                              <1> 	houdini				; (the above conditions are for this)
   385                              <1> 	jmp .datanotfound
   386                              <1> @@:
   387                              <1> %else
   388 00000530 7417                <1> 	je .datanotfound		; no, handle as an error -->
   389                              <1> %endif
   390                              <1> 
   391                              <1> %if ELDDATA_PMREQUIRED_STATUS
   392                              <1> 	mov si, relocateddata
   393                              <1> linkdatarelocation build_option_PM
   394                              <1> 	test si, si			; is it a PM build ?
   395                              <1> 	jz @F				; no --> (treat PM required as optional)
   396                              <1> 	test byte [bp + ?optional], 2	; optional status is PM required ?
   397                              <1> 	jnz .datanotfound		; yes, handle as an error -->
   398                              <1> @@:
   399                              <1> %endif
   400                              <1> 
   401                              <1> %if _ELD_LINKER_PASSES
   402 00000532 36F606[0000]02      <1> 	testopt [ss:relocateddata], 2	; debug optional link ?
   403                              <1> linkdatarelocation options7, -3
   404 00000538 7406                <1> 	jz @F				; no -->
   405 0000053A BE[190B]            <1> 	mov si, lmsg.warning_data_optional
   406                              <1> internalcoderelocation
   407 0000053D E82B00              <1> 	call .notfound			; display a warning
   408                              <1> @@:
   409                              <1> %endif
   410 00000540 E8DBFF              <1> 	call .address_data_reloc
   411 00000543 832400              <1> 	and word [si], 0		; indicate optional data link failed
   412 00000546 E966FF              <1> 	jmp .datarelocloop
   413                              <1> 
   414                              <1> 
   415                              <1> %if _ELDCALL_OPTIONAL
   416                              <1> .coderelocnotfound:
   417                              <1> 	mov byte [si], dl		; restore the original byte at counter
   418                              <1> 	cmp byte [bp + ?optional], 0	; is it an optional relocation ?
   419                              <1> %if _ELD_DEBUG
   420                              <1> 	jne @F
   421                              <1>  %ifn _ELD_LINKER_PASSES
   422                              <1> 	mov si, 0			; (invalid link)
   423                              <1> linkdatarelocation internalflags6
   424                              <1> 	test si, si
   425                              <1> 	jz .codenotfound
   426                              <1> 	mov si, 0			; (invalid link)
   427                              <1> linkdatarelocation options7
   428                              <1> 	test si, si
   429                              <1> 	jz .codenotfound
   430                              <1>  %else
   431                              <1> 	cmp byte [bp + ?pass], 0
   432                              <1> 	je .codenotfound
   433                              <1>  %endif
   434                              <1> 	houdini				; (the above conditions are for this)
   435                              <1> 	jmp .codenotfound
   436                              <1> @@:
   437                              <1> %else
   438                              <1> 	je .codenotfound		; no, handle as an error -->
   439                              <1> %endif
   440                              <1> 
   441                              <1> %if ELDCALL_PMREQUIRED_STATUS
   442                              <1>  %if _ELD_LINKER_PASSES
   443                              <1>   %assign ELDLINKER 0
   444                              <1>  %endif
   445                              <1> 	mov si, relocateddata
   446                              <1> linkdatarelocation build_option_PM
   447                              <1>  %if _ELD_LINKER_PASSES
   448                              <1>   %assign ELDLINKER 1
   449                              <1>  %endif
   450                              <1> 	test si, si			; is it a PM build ?
   451                              <1> 	jz @F				; no --> (treat PM required as optional)
   452                              <1> 	test byte [bp + ?optional], 2	; optional status is PM required ?
   453                              <1> 	jnz .codenotfound		; yes, handle as an error -->
   454                              <1> @@:
   455                              <1> %endif
   456                              <1> 
   457                              <1> %if _ELD_LINKER_PASSES
   458                              <1> 	testopt [ss:relocateddata], 2	; debug optional link ?
   459                              <1> linkdatarelocation options7, -3
   460                              <1> 	jz @F				; no -->
   461                              <1> 	mov si, lmsg.warning_code_optional
   462                              <1> internalcoderelocation
   463                              <1> 	call .notfound			; display a warning
   464                              <1> @@:
   465                              <1> %endif
   466                              <1> 	lds si, [bp + ?entry]		; -> code site (must be in ELD cs)
   467                              <1> 	mov word [si], 9090h
   468                              <1> 	mov byte [si + 2], 90h		; indicate optional code link failed
   469                              <1> 					;  (NOP out the 3-byte call near imm)
   470                              <1> 	jmp .coderelocloop
   471                              <1> %endif
   472                              <1> 
   473                              <1> 
   474                              <1> %if _ELD_LINKER_PASSES
   475                              <1> .datanotfound:
   476 00000549 BE[3B0B]            <1> 	mov si, lmsg.error_data
   477                              <1> internalcoderelocation
   478 0000054C E81C00              <1> 	call .notfound			; display error
   479 0000054F 7203E91F01          <1> 	jnc .error_j			; NC if in pass 0, error out now -->
   480 00000554 FF46E8              <1> 	inc word [bp + ?amounterrors]	; count the amount of errors
   481 00000557 E955FF              <1> 	jmp .datarelocloop		; go to next relocation entry -->
   482                              <1> 
   483                              <1> .codenotfound:
   484 0000055A BE[540B]            <1> 	mov si, lmsg.error_code
   485                              <1> internalcoderelocation
   486 0000055D E80B00              <1> 	call .notfound			; display error
   487 00000560 7203E90E01          <1> 	jnc .error_j			; NC if in pass 0 -->
   488 00000565 FF46E8              <1> 	inc word [bp + ?amounterrors]	; count the amount of errors
   489 00000568 E98400              <1> 	jmp .coderelocloop		; go to next -->
   490                              <1> 
   491                              <1> .notfound:
   492 0000056B 807EEA00            <1> 	cmp byte [bp + ?pass], 0q	; pass 0 ?
   493 0000056F 743A                <1> 	je @F				; yes, do not try displaying --> (NC)
   494 00000571 16                  <1> 	 push ss
   495 00000572 07                  <1> 	 pop es
   496 00000573 BF[0000]            <1> 	mov di, relocateddata
   497                              <1> linkdatarelocation line_out		; es:di -> line_out buffer
   498 00000576 E83300              <1> 	call .copy			; copy prefix message
   499 00000579 8B76E6              <1> 	mov si, word [bp + ?name]
   500 0000057C AD                  <1> 	lodsw				; = hash
   501 0000057D E8[0000]EB020000    <1> 	extcall hexword			; display the hash in hex
   502 00000584 56                  <1> 	push si
   503 00000585 BE[6D0B]            <1> 	mov si, lmsg.error.2
   504                              <1> internalcoderelocation
   505 00000588 E82100              <1> 	call .copy			; display message fragment
   506 0000058B 5E                  <1> 	pop si
   507                              <1> %if _ELD_LINKER_PASSES
   508 0000058C 56                  <1> 	push si
   509 0000058D E81C00              <1> 	call .copy			; copy over the full name
   510 00000590 5E                  <1> 	pop si
   511 00000591 C60400              <1> 	mov byte [si], 0		; mark as failed (counter byte = 0)
   512                              <1> %else
   513                              <1> 	call .copy
   514                              <1> %endif
   515 00000594 B022                <1> 	mov al, '"'
   516 00000596 AA                  <1> 	stosb				; end message with a closing quote mark
   517 00000597 16                  <1> 	 push ss
   518 00000598 1F                  <1> 	 pop ds
   519 00000599 E8[0000]EB020000    <1> 	extcall putsline_crlf		; display diagnostic line
   520 000005A0 B8350E              <1> 	mov ax, 0E35h
   521 000005A3 E8[0000]EB020000    <1> 	extcall setrc
   522 000005AA F9                  <1> 	stc				; CY, diagnostic displayed
   523                              <1> @@:
   524 000005AB C3                  <1> 	retn
   525                              <1> 
   526                              <1> .copy:		; (cannot use extcallcall here)
   527 000005AC E8[0000]EB020000    <1> 	extcall copy_single_counted_string
   528 000005B3 C3                  <1> 	retn
   529                              <1> %else
   530                              <1> .datanotfound: equ .error_j
   531                              <1> .codenotfound: equ .error_j
   532                              <1> %endif
   533                              <1> 
   534                              <1> .build_match:
   535                              <1> %if _ELD_CODE_VSTART
   536 000005B4 2D[0000]            <1> 	sub ax, code			; revert adjustment (= displacement)
   537                              <1> %endif
   538 000005B7 0346FC              <1> 	add ax, word [bp + ?instance]	; make displacement into -> name string
   539 000005BA 96                  <1> 	xchg si, ax			; si -> hash word, counted name string
   540                              <1> %if _ELD_LINKER_PASSES
   541 000005BB 8976E6              <1> 	mov word [bp + ?name], si	; save away for diagnostics
   542                              <1> %endif
   543 000005BE AD                  <1> 	lodsw			; = hash, si -> counted string
   544 000005BF 8A14                <1> 	mov dl, byte [si]	; dl = original start byte of match
   545                              <1> %if _ELD_LINKER_PASSES
   546 000005C1 84D2                <1> 	test dl, dl		; marked as already failed ?
   547 000005C3 750A                <1> 	jnz @F
   548 000005C5 837EE800            <1> 	cmp word [bp + ?amounterrors], 0
   549                              <1> 				; validate error status
   550 000005C9 7503E9A500          <1> 	je .error_j		; no error known ?! cancel quickly -->
   551 000005CE C3                  <1> 	retn			; (NC)
   552                              <1> 
   553                              <1> @@:
   554                              <1> %endif
   555                              <1> %if ELDOTHER
   556                              <1> 	rol byte [bp + ?other], 1
   557                              <1> 	jnc @F
   558                              <1> 	rol byte [bp + ?use_hash_other], 1
   559                              <1> 	jmp @FF
   560                              <1> 
   561                              <1> @@:
   562                              <1> %endif
   563 000005CF D046EC              <1> 	rol byte [bp + ?use_hash], 1
   564                              <1> @@:
   565                              <1> 		; If to use the hash, then ax = hash and si ->
   566                              <1> 		;  the entire symbol name as a counted string.
   567 000005D2 720A                <1> 	jc @F			; if to use hash, return now -->
   568 000005D4 AC                  <1> 	lodsb			; al = length
   569 000005D5 91                  <1> 	xchg cx, ax		; cl = length
   570 000005D6 AD                  <1> 	lodsw			; ax = prefix
   571 000005D7 49                  <1> 	dec cx
   572 000005D8 49                  <1> 	dec cx			; cl = adjusted length
   573 000005D9 4E                  <1> 	dec si			; -> second byte of prefix
   574 000005DA 8A14                <1> 	mov dl, byte [si]	; dl = original start byte of match
   575 000005DC 880C                <1> 	mov byte [si], cl	; si -> counted string suffix
   576                              <1> 		; (this name entry has been edited to provide the
   577                              <1> 		;  name suffix as a counted string, as required by
   578                              <1> 		;  the old-style non-hash link info tables.
   579                              <1> 		; it will be reset later by writing dl to si -> the
   580                              <1> 		;  first byte of the match string.)
   581                              <1> @@:
   582                              <1> %if _ELD_LINKER_PASSES
   583 000005DE F9                  <1> 	stc			; CY
   584                              <1> %endif
   585 000005DF C3                  <1> 	retn
   586                              <1> 
   587                              <1> 
   588                              <1> .donedatareloc:
   589                              <1> %if ELDOTHER
   590                              <1> 	rol byte [bp + ?other], 1
   591                              <1> 	jc .otherdone		; other link only has data links,
   592                              <1> 				;  so at this point we're done -->
   593                              <1> %endif
   594                              <1> 
   595 000005E0 8B56FC              <1> 	mov dx, word [bp + ?instance]
   596                              <1> %if _ELD_LINKER_PASSES
   597 000005E3 8B5EEA              <1> 	mov bx, word [bp + ?pass]
   598 000005E6 01D3                <1> 	add bx, dx
   599                              <1>  %if _ELD_IDENTICALISE
   600                              <1> 	add bx, word [bp + ?lt]
   601                              <1> 	add dx, word [ltLinkCode + bx]
   602                              <1>  %else
   603 000005E8 0397C807            <1> 	add dx, word [linktable - code + ltLinkCode + bx]
   604                              <1>  %endif
   605                              <1> %else
   606                              <1> 	add dx, linkercoderelocations - code
   607                              <1> %endif
   608 000005EC 8956F2              <1> 	mov word [bp + ?nextreloc], dx
   609                              <1> 
   610                              <1> .coderelocloop:
   611 000005EF C576F2              <1> 	lds si, [bp + ?nextreloc]
   612 000005F2 AD                  <1> 	lodsw
   613                              <1> %if _ELDCALL_OPTIONAL
   614                              <1> 	dec ax				; optional word is 1-based, get 0-based
   615                              <1> 	js .donecodereloc
   616                              <1> 	mov word [bp + ?targetsection_low_optional_high], ax
   617                              <1> 	lodsw
   618                              <1> %endif
   619 000005F3 0346FC              <1> 	add ax, word [bp + ?instance]
   620 000005F6 8946EE              <1> 	mov word [bp + ?entry], ax
   621 000005F9 AD                  <1> 	lodsw
   622 000005FA 8976F2              <1> 	mov word [bp + ?nextreloc], si
   623                              <1> %ifn _ELDCALL_OPTIONAL
   624 000005FD 85C0                <1> 	test ax, ax			; if no optional word, check -> match
   625 000005FF 7503E98100          <1> 	jz .donecodereloc
   626                              <1> %endif
   627 00000604 E8ADFF              <1> 	call .build_match
   628                              <1> %if _ELD_LINKER_PASSES
   629 00000607 73E6                <1> 	jnc .coderelocloop
   630                              <1> %endif
   631 00000609 C45EF6              <1> 	les bx, [bp + ?linkinfo]
   632 0000060C 268B4F10            <1> 	mov cx, word [es:bx + eldlCodeAmount]	; amount code link info
   633 00000610 268B7F12            <1> 	mov di, word [es:bx + eldlCodePrefixes]	; -> prefixes or hashes
   634                              <1> .coderelocfind:
   635 00000614 83F901              <1> 	cmp cx, 1			; NZ if cx == 0
   636 00000617 F2AF                <1> 	repne scasw			; scan initial
   637                              <1> %if _ELDCALL_OPTIONAL
   638                              <1> 	jne .coderelocnotfound
   639                              <1> %else
   640                              <1>  %if _ELD_DEBUG
   641                              <1> 	je @F
   642                              <1> 	houdini
   643                              <1> 	jmp .codenotfound
   644                              <1> @@:
   645                              <1>  %else
   646 00000619 7403E93CFF          <1> 	jne .codenotfound
   647                              <1>  %endif
   648                              <1> %endif
   649 0000061E 57                  <1> 	push di
   650 0000061F 51                  <1> 	push cx
   651 00000620 56                  <1> 	push si
   652 00000621 262B7F12            <1> 	sub di, word [es:bx + eldlCodePrefixes]	; = double index, 1-based
   653 00000625 4F                  <1> 	dec di
   654 00000626 4F                  <1> 	dec di				; 0-based
   655 00000627 26037F14            <1> 	add di, word [es:bx + eldlCodeEntries]	; -> entry
   656 0000062B 268B3D              <1> 	mov di, [es:di]			; -> counted suffix/string
   657 0000062E B500                <1> 	mov ch, 0
   658 00000630 8A0C                <1> 	mov cl, byte [si]		; cx = length
   659 00000632 41                  <1> 	inc cx
   660                              <1> 	; cmp al, al			; ZR if length is zero
   661 00000633 F3A6                <1> 	repe cmpsb			; match ?
   662 00000635 5E                  <1> 	pop si
   663 00000636 59                  <1> 	pop cx
   664 00000637 5F                  <1> 	pop di
   665 00000638 75DA                <1> 	jne .coderelocfind
   666 0000063A 8814                <1> 	mov byte [si], dl
   667 0000063C 262B7F12            <1> 	sub di, word [es:bx + eldlCodePrefixes]	; = double index, 1-based
   668 00000640 4F                  <1> 	dec di
   669 00000641 4F                  <1> 	dec di				; 0-based
   670 00000642 01FF                <1> 	add di, di			; quadruple index
   671 00000644 26037F16            <1> 	add di, word [es:bx + eldlCodeAddresses]	; -> address (offset, segment)
   672 00000648 26FF35              <1> 	push word [es:di]
   673 0000064B C576EE              <1> 	lds si, [bp + ?entry]
   674 0000064E 8F4405              <1> 	pop word [si + 3 + 2]		; call near imm (3), jmp short (2)
   675                              <1> 					;  patch the destination address
   676 00000651 803CE8              <1> 	cmp byte [si], 0E8h		; is it as expected ?
   677 00000654 751D                <1> 	jne .error_j
   678 00000656 268B7D02            <1> 	mov di, word [es:di + 2]
   679 0000065A BB[0000]            <1> 	mov bx, relocateddata
   680                              <1> linkdatarelocation linkcall_table	; ss:bx -> link call table
   681 0000065D 36833F01            <1> 	cmp word [ss:bx], 1		; is it initialised to format 1 ?
   682 00000661 7510                <1> 	jne .error_j			; no -->
   683 00000663 368B4F02            <1> 	mov cx, word [ss:bx + 2]	; get amount of segments
   684 00000667 E30A                <1> 	jcxz .error_j			; none -->
   685                              <1> @@:
   686 00000669 83C304              <1> 	add bx, 4			; -> next segment
   687 0000066C 36393F              <1> 	cmp word [ss:bx], di		; value matches ?
   688 0000066F 7405                <1> 	je @F				; yes, found -->
   689 00000671 E2F6                <1> 	loop @B				; try remaining segments
   690                              <1> .error_j:
   691 00000673 E98A00              <1> 	jmp .error
   692                              <1> 
   693                              <1> @@:
   694 00000676 368B5F02            <1> 	mov bx, word [ss:bx + 2]	; -> call destination offset
   695                              <1> 		; si + 3 + delta = bx
   696                              <1> 		; delta = bx - si - 3
   697 0000067A 29F3                <1> 	sub bx, si
   698 0000067C 83EB03              <1> 	sub bx, 3
   699 0000067F 895C01              <1> 	mov word [si + 1], bx		; patch the call instruction
   700 00000682 E96AFF              <1> 	jmp .coderelocloop
   701                              <1> 
   702                              <1> .donecodereloc:
   703                              <1> %if _ELD_LINKER_PASSES
   704 00000685 8B46E8              <1> 	mov ax, word [bp + ?amounterrors]
   705 00000688 85C0                <1> 	test ax, ax
   706 0000068A 75E7                <1> 	jnz .error_j
   707 0000068C 8B5EEA              <1> 	mov bx, word [bp + ?pass]
   708 0000068F 85DB                <1> 	test bx, bx
   709 00000691 750B                <1> 	jnz @F
   710 00000693 43                  <1> 	inc bx
   711 00000694 43                  <1> 	inc bx
   712 00000695 895EEA              <1> 	mov word [bp + ?pass], bx
   713 00000698 8B56FC              <1> 	mov dx, word [bp + ?instance]
   714 0000069B E98DFD              <1> 	jmp .pass
   715                              <1> 
   716                              <1> @@:
   717                              <1> %endif
   718                              <1> 
   719                              <1> %ifnidni _LISTING, ""
   720                              <1> %assign ELDLINKER 0
   721                              <1> .hint:
   722 0000069E 16                  <1> 	push ss
   723 0000069F 1F                  <1> 	pop ds
   724 000006A0 B02D                <1> 	mov al, 2Dh
   725 000006A2 E8[0000]EB020000    <1> 	extcall intchk			; ZR if offset = -1 or segment = 0
   726                              <1> 					; CHG: ax, dx, bx
   727 000006A9 7437                <1> 	jz .no_hint
   728                              <1> 
   729 000006AB 8A26[0000]          <1> 	mov ah, byte [relocateddata]
   730                              <1> linkdatarelocation try_debugger_amis_multiplex_number
   731 000006AF E85500              <1> 	call plex_check
   732 000006B2 7305                <1> 	jnc @F
   733                              <1> 
   734 000006B4 B4FF                <1> 	mov ah, 0FFh		; start with multiplex number 0FFh
   735                              <1> .loop_hint:
   736 000006B6 E84E00              <1> 	call plex_check
   737                              <1> @@:
   738 000006B9 7307                <1> 	jnc .end_hint		; if found --> (NC)
   739 000006BB 80EC01              <1> 	sub ah, 1		; search is backward (to find latest installed first), from 0FFh to 00h including
   740 000006BE 73F6                <1> 	jnc .loop_hint		; try next if we didn't check all yet -->
   741 000006C0 EB20                <1> 	jmp .no_hint
   742                              <1> 
   743                              <1> .end_hint:
   744 000006C2 50                  <1> 	push ax
   745 000006C3 C446FC              <1> 	les ax, [bp + ?instance]
   746 000006C6 BF[0E09]            <1> 	mov di, listmsg.hint.offset
   747                              <1> internalcoderelocation
   748 000006C9 E8[0000]EB020000    <1> 	extcall hexword
   749 000006D0 BB[EC08]            <1> 	mov bx, listmsg.hint
   750                              <1> internalcoderelocation
   751 000006D3 368B16[0000]        <1> 	mov dx, [ss:relocateddata]
   752                              <1> linkdatarelocation extseg	; must be 86 Mode segment even in PM
   753 000006D8 58                  <1> 	pop ax
   754 000006D9 B040                <1> 	mov al, 40h		; AMIS message display service
   755 000006DB E8[0000]EB020000    <1> 	extcall call_int2D
   756                              <1> .no_hint:
   757                              <1> %endif
   758                              <1> 
   759                              <1> %if ELDOTHER
   760                              <1> %assign ELDLINKER 0
   761                              <1> 	not byte [bp + ?other]
   762                              <1> 
   763                              <1> 	push ss
   764                              <1> 	pop ds
   765                              <1> 	mov al, 2Dh
   766                              <1> 	extcall intchk			; ZR if offset = -1 or segment = 0
   767                              <1> 					; CHG: ax, dx, bx
   768                              <1> 	jz .no_other
   769                              <1> 
   770                              <1> 	mov ah, byte [relocateddata]
   771                              <1> linkdatarelocation try_debugger_amis_multiplex_number
   772                              <1> 	call plex_check
   773                              <1> 	jnc @F
   774                              <1> 
   775                              <1> 	mov ah, 0FFh		; start with multiplex number 0FFh
   776                              <1> .loop_other:
   777                              <1> 	call plex_check
   778                              <1> @@:
   779                              <1> 	jnc .end_other		; if found --> (NC)
   780                              <1> 	sub ah, 1		; search is backward (to find latest installed first), from 0FFh to 00h including
   781                              <1> 	jnc .loop_other		; try next if we didn't check all yet -->
   782                              <1> 	jmp .no_other
   783                              <1> 
   784                              <1> .end_other:
   785                              <1> 	mov al, 42h		; AMIS get other link info service
   786                              <1> 	extcall call_int2D
   787                              <1> 	cmp al, 0FFh
   788                              <1> 	jne .no_other
   789                              <1> 
   790                              <1> 	mov ax, si		; selector => PSP
   791                              <1> 	extcall ispm
   792                              <1> 	jz @F
   793                              <1> 	mov ax, dx		; segment => PSP
   794                              <1> @@:
   795                              <1> 	 push ss
   796                              <1> 	 pop ds
   797                              <1> 	mov word [otherds], ax
   798                              <1> internaldatarelocation		; current mode sel/seg
   799                              <1> 	mov word [otherseg], dx
   800                              <1> internaldatarelocation		; remember segment
   801                              <1> 
   802                              <1> 	mov ax, cx		; selector => link info
   803                              <1> 	extcall ispm
   804                              <1> 	jz @F
   805                              <1> 	mov ax, bx		; segment => link info
   806                              <1> @@:
   807                              <1> 	mov word [bp + ?linkinfo_other], di
   808                              <1> 	mov word [bp + ?linkinfo_other + 2], ax
   809                              <1> 
   810                              <1> 	mov ds, ax		; => link info
   811                              <1> 	xor ax, ax
   812                              <1> 	cmp word [di + eldlSignature], 0E1D1h
   813                              <1> 	jne .error_other
   814                              <1> 	cmp word [di + eldlUseLinkHash], 1
   815                              <1> 	ja .error_other
   816                              <1> 	jb @F
   817                              <1> 	dec ax
   818                              <1> @@:
   819                              <1> 	mov word [bp + ?use_hash_other], ax
   820                              <1> 
   821                              <1> 	mov dx, word [bp + ?instance]
   822                              <1> 	add dx, linkerotherdatarelocations - code
   823                              <1> 	jmp .otherloop
   824                              <1> 
   825                              <1> .error_other:
   826                              <1> 	push cs
   827                              <1> 	pop ds
   828                              <1> 	mov ax, 0E33h
   829                              <1> 	extcall setrc
   830                              <1> 	mov dx, lmsg.error_other
   831                              <1> internalcoderelocation
   832                              <1> 	jmp @F
   833                              <1> 
   834                              <1> .no_other:
   835                              <1> 	push cs
   836                              <1> 	pop ds
   837                              <1> 	mov ax, 0E34h
   838                              <1> 	extcall setrc
   839                              <1> 	mov dx, lmsg.no_other
   840                              <1> internalcoderelocation
   841                              <1> @@:
   842                              <1> 	extcall putsz
   843                              <1> .error_j2:
   844                              <1> 	jmp .error
   845                              <1> 
   846                              <1> .otherdone:
   847                              <1>  %if _ELD_LINKER_PASSES
   848                              <1> 	mov ax, word [bp + ?amounterrors]
   849                              <1> 	test ax, ax
   850                              <1> 	jnz .error_j2
   851                              <1>  %endif
   852                              <1> %endif
   853                              <1> 
   854 000006E2 5B                  <1> 	pop bx				; -> our heap data
   855 000006E3 5E                  <1> 	pop si				; -> our command line tail
   856 000006E4 16                  <1> 	 push ss
   857 000006E5 1F                  <1> 	 pop ds
   858 000006E6 C47EFC              <1> 	les di, [bp + ?instance]
   859 000006E9 268B4502            <1> 	mov ax, word [es:di + eldiEndCode]
   860                              <1> houdini
   861 000006ED 2D[0004]            <1> 	sub ax, strict word endresident + code
   862                              <1> internalcoderelocation
   863 000006F0 26C74502[0004]      <1> 	mov word [es:di + eldiEndCode], endresident + code
   864                              <1> internalcoderelocation
   865 000006F6 2906[0000]          <1> 	sub word [relocateddata], ax
   866                              <1> linkdatarelocation extseg_used
   867                              <1> %if _DATA_SIZE == 0
   868                              <1> 	xor ax, ax
   869                              <1> 	mov word [es:di + eldiStartData], ax
   870                              <1> 	mov word [es:di + eldiEndData], ax
   871                              <1> %endif
   872 000006FA 89EC5D              <1> 	lleave code
   873                              <1> 		; INP:	es => ELD code segment
   874                              <1> 		;	ds:si -> command line tail
   875                              <1> 		;	ds:bx -> ELD data block
   876                              <1> 		;	ss:sp -> far return address for current mode
   877                              <1> 		; STT:	ds = ss, UP, EI
   878 000006FD E958FC              <1> 	jmp start
   879                              <1> 
   880                              <1> .error:
   881 00000700 89EC5D              <1> 	lleave
   882 00000703 B8FFFF              <1> 	mov ax, -1
   883 00000706 CB                  <1> 	retf
   884                              <1> 
   885                              <1> 
   886                              <1> %ifnidni _LISTING, ""
   887                              <1>  %assign ELDHINT 1
   888                              <1> %else
   889                              <1>  %assign ELDHINT 0
   890                              <1> %endif
   891                              <1> 
   892                              <1> %if ELDOTHER || ELDHINT
   893                              <1> 		; INP:	ah = multiplex number to check
   894                              <1> 		; OUT:	CY if multiplex number unused or no signature match,
   895                              <1> 		;	 bp, ah, ds unmodified
   896                              <1> 		;	NC if match found,
   897                              <1> 		;	 ah = multiplex number (unmodified)
   898                              <1> 		; CHG:	si, di, es, cx, dx
   899                              <1> plex_check:
   900 00000707 16                  <1> 	push ss
   901 00000708 1F                  <1> 	pop ds
   902 00000709 F606[0000]08        <1> 	testopt [relocateddata], 8
   903                              <1> linkdatarelocation internalflags4, -3
   904 0000070E 740B                <1> 	jz @F
   905 00000710 BE[0000]            <1> 	mov si, relocateddata
   906                              <1> linkdatarelocation amis_multiplex_number, -2, optional
   907 00000713 85F6                <1> 	test si, si
   908 00000715 7404                <1> 	jz @F
   909 00000717 3A24                <1> 	cmp ah, byte [si]
   910 00000719 7420                <1> 	je .notfound		; do not use our own multiplexer -->
   911                              <1> @@:
   912 0000071B B000                <1> 	mov al, 00h		; AMIS installation check
   913 0000071D E8[0000]EB020000    <1> 	extcall call_int2D	; AMIS (or "DOS reserved" = iret if no AMIS present)
   914 00000724 3CFF                <1> 	cmp al, 0FFh
   915 00000726 7513                <1> 	jne .notfound
   916 00000728 0E                  <1> 	push cs
   917 00000729 1F                  <1> 	pop ds
   918 0000072A BE[DC08]            <1> 	mov si, debuggeramissig	; ds:si -> our AMIS name strings
   919                              <1> internalcoderelocation
   920 0000072D E8[0000]EB020000    <1> 	extcall setes2dx	; es:di -> name strings of AMIS multiplexer that just answered
   921 00000734 B90800              <1> 	mov cx, 8		; Ignore description, only compare vendor and program name
   922 00000737 F3A7                <1> 	repe cmpsw
   923 00000739 7401                <1> 	je .checkret		; ZR, NC = match -->
   924                              <1> .notfound:
   925 0000073B F9                  <1> 	stc			; CY no match
   926                              <1> .checkret:
   927 0000073C C3                  <1> 	retn
   928                              <1> %endif
   929                              <1> 
   930                              <1> 
   931 0000073D 00<rep 3h>          <1> 	align 4, db 0
   932                              <1> linkercoderelocations:
   933                              <1> %if _ELDCALL_OPTIONAL
   934                              <1> 	dw ELDCALL_CODE_RELOCATIONS_OPTIONAL, 0
   935                              <1> %else
   936 00000740 2200[1609]6A00-     <1> 	dw ELDCALL_CODE_RELOCATIONS, 0, 0
   936 00000746 [2509]FD01[2509]F0- <1>
   936 0000074D 02[3509]F802[4109]- <1>
   936 00000754 0003[4D09]0803-     <1>
   936 0000075A [5609]1003[5D09]18- <1>
   936 00000761 03[6609]2003[7209]- <1>
   936 00000768 2803[7E09]3003-     <1>
   936 0000076E [8E09]3803[9809]40- <1>
   936 00000775 03[A009]4803[A809]- <1>
   936 0000077C 5003[B009]6B03-     <1>
   936 00000782 [A009]9C03[4D09]A2- <1>
   936 00000789 06[EE09]C906[B709]- <1>
   936 00000790 DB06[F709]1D07-     <1>
   936 00000796 [F709]2D07[040A]00- <1>
   936 0000079D 000000              <1>
   937                              <1> %endif
   938                              <1> 
   939                              <1> %if _ELD_LINKER_PASSES
   940                              <1> linkerlinkercoderelocations:
   941                              <1> %if _ELDCALL_OPTIONAL
   942                              <1> 	dw ELDCALL_LINKER_CODE_RELOCATIONS_OPTIONAL, 0
   943                              <1> %else
   944 000007A0 7D05[B709]9905-     <1> 	dw ELDCALL_LINKER_CODE_RELOCATIONS, 0, 0
   944 000007A6 [C109]A305[A809]AC- <1>
   944 000007AD 05[D109]00000000    <1>
   945                              <1> %endif
   946                              <1> 
   947                              <1> 	align 2, db 0
   948                              <1> linktable:
   949                              <1> 	istruc LINKTABLE
   950                              <1> at ltCodeToCode
   951 000007B4 CC08                <1> 	dw internallinkercodetocoderelocations - code
   952 000007B6 4608                <1> 	dw internalcodetocoderelocations - code
   953                              <1> at ltCodeToData
   954 000007B8 D608                <1> 	dw internallinkercodetodatarelocations - code
   955 000007BA 6808                <1> 	dw internalcodetodatarelocations - code
   956                              <1> at ltDataToCode
   957 000007BC D808                <1> 	dw internallinkerdatatocoderelocations - code
   958 000007BE A008                <1> 	dw internaldatatocoderelocations - code
   959                              <1> at ltDataToData
   960 000007C0 DA08                <1> 	dw internallinkerdatatodatarelocations - code
   961 000007C2 A608                <1> 	dw internaldatatodatarelocations - code
   962                              <1> at ltLinkData
   963 000007C4 B808                <1> 	dw linkerlinkerdatarelocations - code
   964 000007C6 CC07                <1> 	dw linkerdatarelocations - code
   965                              <1> at ltLinkCode
   966 000007C8 A007                <1> 	dw linkerlinkercoderelocations - code
   967 000007CA 4007                <1> 	dw linkercoderelocations - code
   968                              <1> 	iend
   969                              <1> %endif
   970                              <1> 
   971                              <1> 	align 2, db 0
   972                              <1> linkerdatarelocations:
   973 000007CC 01004700[0F0A]0100- <1> 	dw LINK_DATA_RELOCATIONS, 0
   973 000007D4 4900[190A]01004C00- <1>
   973 000007DC [220A]01006701-     <1>
   973 000007E2 [320A]0100DD02-     <1>
   973 000007E8 [3C0A]0100E602-     <1>
   973 000007EE [470A]01006103-     <1>
   973 000007F4 [500A]01007B03-     <1>
   973 000007FA [5E0A]01008B03-     <1>
   973 00000800 [690A]01009803-     <1>
   973 00000806 [770A]02000200-     <1>
   973 0000080C [860A]02000800-     <1>
   973 00000812 [990A]0100AF03-     <1>
   973 00000818 [690A]0100BB03-     <1>
   973 0000081E [770A]0100F003-     <1>
   973 00000824 [5E0A]0100AD06-     <1>
   973 0000082A [CB0A]0100D606-     <1>
   973 00000830 [470A]0100F806-     <1>
   973 00000836 [690A]01000B07-     <1>
   973 0000083C [F00A]01011107-     <1>
   973 00000842 [010B]0000          <1>
   974                              <1> 
   975                              <1> 	align 2, db 0
   976                              <1> internalcodetocoderelocations:
   977 00000846 DF01F5010B02BF0282- <1> 	dw INTERNAL_CODE_TO_CODE_RELOCATIONS, 0
   977 0000084F 0387038F039403AB03- <1>
   977 00000858 B703EB03C706D106EE- <1>
   977 00000861 06F4062B070000      <1>
   978                              <1> 
   979                              <1> 	align 2, db 0
   980                              <1> internalcodetodatarelocations:
   981 00000868 340057007D00820087- <1> 	dw INTERNAL_CODE_TO_DATA_RELOCATIONS, 0
   981 00000871 00AC00450153016001- <1>
   981 0000087A 72017A018801BE01C5- <1>
   981 00000883 01E901ED0115021C02- <1>
   981 0000088C 3A024902B902C302D7- <1>
   981 00000895 026903BE03E403F603- <1>
   981 0000089E 0000                <1>
   982                              <1> 
   983                              <1> 	align 2, db 0
   984                              <1> internaldatatocoderelocations:
   985 000008A0 00000600FFFF        <1> 	dw INTERNAL_DATA_TO_CODE_RELOCATIONS, -1
   986                              <1> 
   987                              <1> 	align 2, db 0
   988                              <1> internaldatatodatarelocations:
   989 000008A6 0C000E001000120018- <1> 	dw INTERNAL_DATA_TO_DATA_RELOCATIONS, -1
   989 000008AF 001A001C001E00FFFF  <1>
   990                              <1> 
   991                              <1> %if _ELD_LINKER_PASSES
   992                              <1> 	align 2, db 0
   993                              <1> linkerlinkerdatarelocations:
   994 000008B8 01003505[5E0A]0100- <1> 	dw LINK_LINKER_DATA_RELOCATIONS, 0
   994 000008C0 7405[AF0A]01005B06- <1>
   994 000008C8 [BA0A]0000          <1>
   995                              <1> 
   996                              <1> 	align 2, db 0
   997                              <1> internallinkercodetocoderelocations:
   998 000008CC 3B054A055B05860500- <1> 	dw INTERNAL_LINKER_CODE_TO_CODE_RELOCATIONS, 0
   998 000008D5 00                  <1>
   999                              <1> 
  1000                              <1> 	align 2, db 0
  1001                              <1> internallinkercodetodatarelocations:
  1002 000008D6 0000                <1> 	dw INTERNAL_LINKER_CODE_TO_DATA_RELOCATIONS, 0
  1003                              <1> 
  1004                              <1> 	align 2, db 0
  1005                              <1> internallinkerdatatocoderelocations:
  1006 000008D8 FFFF                <1> 	dw INTERNAL_LINKER_DATA_TO_CODE_RELOCATIONS, -1
  1007                              <1> 
  1008                              <1> 	align 2, db 0
  1009                              <1> internallinkerdatatodatarelocations:
  1010 000008DA FFFF                <1> 	dw INTERNAL_LINKER_DATA_TO_DATA_RELOCATIONS, -1
  1011                              <1> %endif
  1012                              <1> 
  1013                              <1> %if ELDOTHER
  1014                              <1> 	align 2, db 0
  1015                              <1> linkerotherdatarelocations:
  1016                              <1> 	dw LINK_OTHER_DATA_RELOCATIONS, 0
  1017                              <1> 
  1018                              <1>  %ifnidn LINK_OTHER_LINKER_DATA_RELOCATIONS, ""
  1019                              <1>   %error Other linker data links not supported
  1020                              <1>  %endif
  1021                              <1> %endif
  1022                              <1> 
  1023                              <1> %if ELDOTHER || ELDHINT
  1024                              <1> 	align 2, db 0
  1025                              <1> debuggeramissig:
  1026 000008DC 65636D20<rep 5h>    <1> 		fill 8, 32, db "ecm"
  1027 000008E4 6C446562756720-     <1> 		fill 8, 32, db "lDebug"
  1027 000008E4 <rep 2h>            <1>
  1028                              <1> %endif
  1029                              <1> 
  1030                              <1> %ifnidni _LISTING, ""
  1031                              <1> listmsg:
  1032 000008EC 547261634C6973742D- <1> .hint:		db "TracList-add-offset=",_LISTING,"::"
  1032 000008F5 6164642D6F66667365- <1>
  1032 000008FE 743D75736570617261- <1>
  1032 00000907 742E6C73743A3A      <1>
  1033 0000090E 2D2D2D2D680D0A00    <1> .hint.offset:	asciz "----h",13,10
  1034                              <1> %endif
  1035                              <1> 
  1036 00000916 30CD0C636D64335F6E- <1> 	eldcall_dump_names ELDCALL_CODE_NAMES
  1036 0000091F 6F745F6578741AB70D- <1>
  1036 00000928 707574735F6578745F- <1>
  1036 00000931 646F6E65D55509736B- <1>
  1036 0000093A 6970636F6D6D6103C3- <1>
  1036 00000943 096973737472696E67- <1>
  1036 0000094C 3FDDB90663686B656F- <1>
  1036 00000955 6CBABD04636D643322- <1>
  1036 0000095E 10066765746E796229- <1>
  1036 00000967 EF09736B6970776869- <1>
  1036 00000970 7465A45509736B6970- <1>
  1036 00000979 636F6D6D308B1E0D70- <1>
  1036 00000982 7574735F6578745F6E- <1>
  1036 0000098B 6578743D8207676574- <1>
  1036 00000994 62797465A7AA056572- <1>
  1036 0000099D 726F72551205707574- <1>
  1036 000009A6 737AB2120573657472- <1>
  1036 000009AF 632890046973706D84- <1>
  1036 000009B8 8107686578776F7264- <1>
  1036 000009C1 6FA20D707574736C69- <1>
  1036 000009CA 6E655F63726C66D0BB- <1>
  1036 000009D3 1A636F70795F73696E- <1>
  1036 000009DC 676C655F636F756E74- <1>
  1036 000009E5 65645F737472696E67- <1>
  1036 000009EE 986906696E7463686B- <1>
  1036 000009F7 21300A63616C6C5F69- <1>
  1036 00000A00 6E743244B774087365- <1>
  1036 00000A09 746573326478        <1>
  1037 00000A0F C30B076C617374636D- <1> 	link_data_dump_names LINK_DATA_NAMES
  1037 00000A18 646B5D06646D79636D- <1>
  1037 00000A21 6454400D6D73672E75- <1>
  1037 00000A2A 6E696E7374616C6C10- <1>
  1037 00000A33 32077265675F656178- <1>
  1037 00000A3C EB4208657874647373- <1>
  1037 00000A45 656CD52D0665787473- <1>
  1037 00000A4E 65678D710B6D73672E- <1>
  1037 00000A57 696E7374616C6C5ABC- <1>
  1037 00000A60 086F7074696F6E7337- <1>
  1037 00000A69 E7D30B657874736567- <1>
  1037 00000A72 5F75736564B2400C65- <1>
  1037 00000A7B 7874646174615F7573- <1>
  1037 00000A84 6564AE24106578745F- <1>
  1037 00000A8D 707574735F68616E64- <1>
  1037 00000A96 6C657297B613657874- <1>
  1037 00000A9F 5F636F6D6D616E645F- <1>
  1037 00000AA8 68616E646C657284E3- <1>
  1037 00000AB1 086C696E655F6F7574- <1>
  1037 00000ABA 68440E6C696E6B6361- <1>
  1037 00000AC3 6C6C5F7461626C65F0- <1>
  1037 00000ACC 9E227472795F646562- <1>
  1037 00000AD5 75676765725F616D69- <1>
  1037 00000ADE 735F6D756C7469706C- <1>
  1037 00000AE7 65785F6E756D626572- <1>
  1037 00000AF0 CB510E696E7465726E- <1>
  1037 00000AF9 616C666C6167733468- <1>
  1037 00000B02 8C15616D69735F6D75- <1>
  1037 00000B0B 6C7469706C65785F6E- <1>
  1037 00000B14 756D626572          <1>
  1038                              <1> %if ELDOTHER
  1039                              <1> 	link_data_dump_names LINK_OTHER_DATA_NAMES
  1040                              <1> %endif
  1041                              <1> 
  1042                              <1> lmsg:
  1043                              <1> %if _ELD_LINKER_PASSES
  1044                              <1> %if _ELDCALL_OPTIONAL
  1045                              <1> .warning_code_optional:		counted "Optional code link missing, hash="
  1046                              <1> %endif
  1047 00000B19 214F7074696F6E616C- <1> .warning_data_optional:		counted "Optional data link missing, hash="
  1047 00000B22 2064617461206C696E- <1>
  1047 00000B2B 6B206D697373696E67- <1>
  1047 00000B34 2C20686173683D      <1>
  1048 00000B3B 1844617461206C696E- <1> .error_data:			counted "Data link missing, hash="
  1048 00000B44 6B206D697373696E67- <1>
  1048 00000B4D 2C20686173683D      <1>
  1049 00000B54 18436F6465206C696E- <1> .error_code:			counted "Code link missing, hash="
  1049 00000B5D 6B206D697373696E67- <1>
  1049 00000B66 2C20686173683D      <1>
  1050 00000B6D 0A682C206C6162656C- <1> .error.2:			counted "h, label ",'"'
  1050 00000B76 2022                <1>
  1051                              <1> %endif
  1052                              <1> %if ELDOTHER
  1053                              <1> .no_other:		asciz "ELD linker: No other link info found!",13,10
  1054                              <1> .error_other:		asciz "ELD linker: Other link info unknown format!",13,10
  1055                              <1> %endif
  1056                              <1> 
  1057 00000B78 00<rep 8h>          <1> 	align 16, db 0
   734                                  
   735                                  	align 16
   736                                  code_size equ $ - code
